S31508001800B00A0020D9180008E7180008E9180008E7
S3150800181000000000000000000000000000000000BA
S315080018200000000000000000000000000119000888
S31508001830000000000000000003190008093B00082A
S31508001840A14B00080719000807190008071900081E
S3150800185007190008071900080719000807190008DA
S31508001860071900089D290008071900080719000824
S3150800187007190008071900080719000807190008BA
S3150800188007190008000000000000000007190008FA
S3150800189000000000071900080719000807190008C2
S315080018A000000000071900080719000895440008F9
S315080018B007190008071900080719000800000000A2
S315080018C0EE11AA550348854600F006FD0048004774
S315080018D0B9790008B00A00200B4880F308880B483D
S315080018E080470B480047FEE704207146084202D0AD
S315080018F0EFF3098001E0EFF30880714605F0A8FED2
S31508001900FEE7FEE7FEE7FEE7B00A0020C13D000855
S31508001910C518000830B50B460146002020220124D0
S3150800192009E00D46D5409D4205D31D469540491B05
S315080019302546954040191546521E002DF1DC30BD4E
S3150800194070B500242546002801DA01244042002902
S3150800195001DA01254942FFF7DDFFAC4200D04042DB
S31508001960002C00D0494270BD03460B439B0703D0A9
S3150800197009E008C9121F08C0042AFAD203E00B7846
S315080019800370401C491C521EF9D27047D2B201E0BE
S315080019900270401C491EFBD270470022F6E710B5BC
S315080019A013460A4604461946FFF7F0FF204610BDBF
S315080019B0F8B502464A40D40F42004B0052085B086D
S315080019C09A4202D20246084611464A0023D0C30D5F
S315080019D04A00DDB2120EAD1A202D35DA490201266B
S315080019E0490AF6058A19002C00D0524220214F1BBD
S315080019F01146B9402A411018C20D9A4221D0002C2E
S31508001A0017D0012D08DCDA05801AD20F8019D20703
S31508001A10DBB200F077FBF8BDDA05801A0123400037
S31508001A201B06C01880185A428018CA0F104349006E
S31508001A3007E04908C2071143DA05801A80194008E9
S31508001A40801800F057FBF8BD61000122511A001BEF
S31508001A50F7E70122D2075140AAE70122D2075040F0
S31508001A60A6E7024670B54A40D30FDB0740002DD0E3
S31508001A704A002AD0010E140E000212020919400A61
S31508001A80520A8418E50104465443000A120A2E0431
S31508001A905043A4194219200CC543AA18120C012553
S31508001AA0AD03521C521912047F39240400D0521C6B
S31508001AB0104301D44000491EC2B20C06C0092018C2
S31508001AC0401C4008802A02D003E0002070BD400870
S31508001AD04000002900DA0020184370BD70B50246A0
S31508001AE04A40D50F40004A00ED0740085208002832
S31508001AF014D0002A12D0C40DD30D41020120C0050E
S31508001B005202490A520AE41A091812187D349142F7
S31508001B1001D3641C00E04900002C01DA002070BDE6
S31508001B200023914201D3891A03434008490000283B
S31508001B30F7D100290AD0914202D10121C90705E04F
S31508001B40914201D2012101E00121C943E005C018F3
S31508001B50401900F0CFFA70BDF0B507460846584060
S31508001B6087B0C00F049048000E465900400849083F
S31508001B70BC1A884105D2384631461E4617460B46DA
S31508001B8002465800400810434CD0300D03904005DB
S31508001B905900400D490D0590401A0290402872DA06
S31508001BA018030121000B09050843019004980092C7
S31508001BB0002805D0019952420020884100920190E0
S31508001BC0029840210A1A0199009800F05FFA054622
S31508001BD00C466B4607CB00F07AFAC0197141039A96
S31508001BE00E0D0023D71756401A467A40164344D09E
S31508001BF0049A002A2DD0029A012A039A15DC1205A6
S31508001C00C01A914101263605001C7141D20F059E66
S31508001C10D2070093019202962A46234600F0B8FAA4
S31508001C2007B0F0BD38463146FAE71605224A0F4690
S31508001C30B218C01AB74101210905001C4F41001806
S31508001C407F41114618187941E20F10436D19644116
S31508001C5013E0E2076D0815436408C2071443039AA4
S31508001C6001261205C01A91413605001C7141CE079E
S31508001C70400830434908C01851412A46234600F017
S31508001C807AFACDE7FFE7049801224000C117121A35
S31508001C9000238B4104983146C417381AA141EEE750
S31508001CA030B40124E407634030BC55E730B401245E
S31508001CB0E407614030BC4FE70000E0FFF0B51FB411
S31508001CC088B00B990998002448400999C00F490023
S31508001CD049080991C0070B990090490049080B91DA
S31508001CE009990898A64608431CD00B990A980843F0
S31508001CF018D0099801244000420D4800410D099862
S31508001D0024050003000B204309900B980003000BE1
S31508001D1020430B9050181C49401800220190144685
S31508001D20104605E0002001460DB0F0BD032801DA93
S31508001D30034600E003239C46C11A0AAE0AE05F0088
S31508001D4008ADED5B4F00F75B7D430027AA187C4181
S31508001D50491C5B1E6145F2DD410004AB5A52210461
S31508001D60120C0A43240C401C0828DFDB0198029059
S31508001D700099704601910090059B049A0799069868
S31508001D8000F006FAD0E700000DFCFFFFF0B50C46A0
S31508001D905C4085B0E40FE40703944C000026640811
S31508001DA059009446490802460296224321D06246C3
S31508001DB00A431ED06200570D4A000E032303550D31
S31508001DC0012402462C492405781B1B0B360B4018A8
S31508001DD023432643614600901C46501AB44103D358
S31508001DE00098401C009002E0921800985B41002879
S31508001DF003DA0020014605B0F0BD002001210905DF
S31508001E000746864611E064461D46141BB54106D3AF
S31508001E106546521BB341744607430C43A646CD0795
S31508001E2040084908284392185B4105460D43EAD104
S31508001E301046184313D0604619465040714008436F
S31508001E4006D06046101AB34106D20122002306E0E6
S31508001E5000220123DB0702E00122D2435310009837
S31508001E6074460105381C6141029C039D00196941AD
S31508001E7000F081F9BFE70000FD030000C217C10F9B
S31508001E80504010B54018CA079623002100F03AF9C9
S31508001E9010BD10B500229623114600F033F910BD87
S31508001EA00EB5C217C10F5040CA0740180021054B8E
S31508001EB00293019200910A460B4600F069F903B0B5
S31508001EC000BD0000330400000EB50549029100214B
S31508001ED000910A460B46019100F05AF903B000BD7D
S31508001EE033040000C20F410040020123400ADB050B
S31508001EF0D207090EC0187F2901DA002070479629F3
S31508001F0003DC9623591AC84001E096398840002A0E
S31508001F10F4D040427047410040020122400AD205EF
S31508001F20090E80187F2901DA00207047962903DCFC
S31508001F309622511AC8407047963988407047000063
S31508001F404A0009030123090B1B051943094B10B560
S31508001F50520D9A4201DA002010BD064B34339A42DC
S31508001F6003DC9A1A00F0A2F810BD034951188840FC
S31508001F7010BD0000FF030000CDFBFFFFC20FD20714
S31508001F80400040080BD0C10D0723DB01C9184002E9
S31508001F900905400A1143C20840071143704700204B
S31508001FA00146704710B5002904DB0124E4074042C6
S31508001FB08C412146002B04DB1C460123DB075242D9
S31508001FC0A3418B4200D1824210BD0000CB0FDB0734
S31508001FD0490010B5490802460A4307D00A0D0724E6
S31508001FE00903E401090B121B002A01DC002010BDBD
S31508001FF0C900440F0C43C100E018D205801800F050
S3150800200079F810BD0122D207002800DB101A002932
S3150800201000DB511A814270470122D207002800DBF3
S31508002020101A002900DB511A88427047F0B51FB410
S315080020300646002082B005464024019100901BE028
S31508002040019922460F46304600F030F8049A059B5F
S31508002050801A994110D310461946224600F016F800
S31508002060361A8F410197224601200021009F00F071
S315080020700DF838184D4100902046641E0028DFDC14
S31508002080019B00982946324607B0F0BD10B5202AB4
S3150800209004DB0146203A9140002010BD91402023E0
S315080020A09C1A0346E3401943904010BD10B5202AF8
S315080020B004DB0846203AD040002110BD0B46D34029
S315080020C0D0402024A21A91400843194610BD10B5E5
S315080020D0202A06DBCB170846203A1041C1170B43C6
S315080020E006E00B461341D0402024A21A914008432B
S315080020F0194610BD002904DA401C490001D14008E0
S315080021004000704770B40024050C05D11024000463
S3150800211002D1002921D01124050E01D1000208346C
S31508002120050F01D10001241D850F01D18000A41CD3
S31508002130002801DB4000641C002908D020252E1B3E
S315080021400D46F540A14000D0012129430843010668
S315080021501B1B000ADB1D02D5002070BC7047DB057F
S31508002160181880180029F8DA401C4900F5D170BC07
S3150800217040084000704710B5002B08DA0024401CC0
S31508002180614192185B411A4301D14008400010BDD5
S31508002190F0B51FB482B005460C0003D0084602F01D
S315080021A085FD02E002F082FD2030024600902146BD
S315080021B02846FFF76BFF049B059A04460F4618430B
S315080021C01143084314D0184610431BD000984021E9
S315080021D00A1A18460599FFF769FF05460E46009A3A
S315080021E005990498FFF752FF084305D0012004E03B
S315080021F02046394607B0F0BD0020C11705430E43F7
S315080022002C43374300990E986305401A7905E40A6A
S3150800221000220C43FD0A0A3002D500200146E9E7F0
S315080022200105101969410C9C0D9D00196941FFF7BC
S31508002230A2FFDFE7FEB500231A461B1A8A4103DB15
S315080022400020014603B0F0BD4A000D0301212D0B05
S315080022500905520D0D43D10702D100186D41521ED2
S315080022605110FF31FF310131002704463E463846FA
S31508002270009701910246012100200905FFF716FF84
S31508002280C3197141F818324684468E464A4161465A
S315080022902846611A904104D36046241A9541764629
S315080022A01F46241900986D41401C00903428E1DD32
S315080022B0F91930467041091BA84103D20022D243BE
S315080022C0134601E00022134601980105381C7141A6
S315080022D0FFF751FFB6E70000064C0125064E05E05C
S315080022E0E36807CC2B430C3C98471034B442F7D329
S315080022F0FFF7ECFAB09A0008D09A000870B58C1867
S315080023000578401C6B075B0F01D10378401C2A1126
S3150800231006D10278401C03E006780E70401C491C62
S315080023205B1EF9D12B0705D40023521E0DD40B7062
S31508002330491CFAE70378401CCB1A921C03E01D7867
S315080023400D70491C5B1C521EF9D5A142D8D300203A
S3150800235070BD000010B50446002C08D101210920E3
S31508002360C00600F0E7FD002000F0E6F852E0012C78
S3150800237005D102210920C00600F0DCFD4AE0022C46
S3150800238005D104210920C00600F0D4FD42E0032C43
S3150800239005D108210920C00600F0CCFD3AE0042C3E
S315080023A005D110210920C00600F0C4FD32E0052C35
S315080023B005D120210920C00600F0BCFD2AE0062C24
S315080023C005D140210920C00600F0B4FD22E0072C03
S315080023D005D180210920C00600F0ACFD1AE0082CC2
S315080023E004D101210D4800F0A5FD13E0092C04D104
S315080023F002210A4800F09EFD0CE00B2C04D11021A6
S31508002400064800F097FD05E00C2C03D1802103480F
S3150800241000F090FD204600F08FF810BD000400483B
S315080024207FB500200090019002900390002427E0D9
S3150800243000250CE0E800294940186100405AA1002F
S315080024406A4651584018A1005050681C85B2142D90
S31508002450F0DBA1006A4650581421FFF75BFA2821E1
S31508002460484361001E4A515A3C225143461864218A
S315080024703046FFF74FFA6100194A5052601C84B281
S31508002480042CD5DB1748807E002826D014484088BF
S315080024901549884203DC1248808888420ADD1148BB
S315080024A02038C079002805D11049486005210D4813
S315080024B02038C1710A4840880A2803DB0848808802
S315080024C00A280ADA07482038C079002805D10749BA
S315080024D04860042103482038C1717FBDF4040020F8
S315080024E0740100202C040020E60F00000C020020D6
S315080024F000B587B001A800F0AFF80121480201F045
S3150800250075F9002001907020029001208002039046
S3150800251000200690059001A9064800F031F801212F
S31508002520044800F021F80121024800F011F807B02C
S3150800253000BD00000024014010B504460723002210
S315080025402146024800F038F810BD0000002401407A
S31508002550002904D0426801231A43426003E0426816
S315080025605208520042607047002904D08268082346
S315080025701A43826003E0826808239A4382607047A0
S3150800258042680B4B1A4042600B684A681A43436814
S315080025901A4342608268074B1A4082600B694A698F
S315080025A01A438B681A4383681A438260704700008F
S315080025B00FBCFFFF8FF1F9FFF0B504460D4616462E
S315080025C01F463F073F0F2B46082B0FD91B071B0F2C
S315080025D0083B606F9A000F21914088436067606FDF
S315080025E099003A468A40104360670BE0206F9A00CC
S315080025F00F21914088432067206F99003A468A4008
S3150800260010432067E0680121A9408843E060E0683C
S315080026100121A9400843E0600120800328400028E2
S3150800262003D0012000F020F807E00120C00328406D
S31508002630002802D0012000F017F8F0BD002905D0C7
S315080026408268FF2301331A43826004E08268FF230D
S3150800265001339A43826070470021016041608160BE
S315080026600173016141617047002806D0064949682F
S315080026700C221143044A516005E0034949680C22BB
S315080026809143014A516070470024014010B524481F
S315080026900078012834D10020214908702149088092
S315080026A012E02048008840001F49085A1F49098837
S315080026B0C9001F4A89181B4A1288520088521948AD
S315080026C00088401C17490880164800880428E8DB5B
S315080026D07E2002F071FA022000F02EF90121154839
S315080026E0FFF7ACFF11480088401C104908800846CF
S315080026F00088142804DB0020088001200E49087091
S315080027000D480078002806D0FFF78AFE00200A49FF
S31508002710087000F059FC7E2002F04EFA10BD000049
S31508002720840100209E010020BC040020A001002096
S31508002730F4040020002401407C010020FFB583B08A
S315080027400C46029400200190002726E000261CE093
S31508002750721C039951430846791CFFF7DBF80546B6
S31508002760A54201D9281B00E0601B05460298A8422D
S3150800277004D90295059806700698077002980028ED
S3150800278002D10120019002E0761C402EE0D300BF62
S315080027900198002800D002E07F1C042FD6D300BF82
S315080027A0029807B0F0BD000000BF00BF00BF00BF21
S315080027B000BFBFF34F8F00BF00BF00BF06480749E1
S315080027C0C86000BF00BF00BFBFF34F8F00BF00BF88
S315080027D000BF00BF00BFFDE70400FA0500ED00E0FA
S315080027E010B500F001F810BD10B523480078002890
S315080027F017D1224801F082F801283CD11F480078F9
S31508002800002838DD1D480078402834DC01F016FE23
S315080028101B490860012018490870002019490870EA
S3150800282029E0164A17490978491C501801F066F834
S31508002830012816D113480078401C124908700F4821
S3150800284000780978884216D100200B4908700B4891
S315080028504078FF280FD10B48007802280BD1FFF7E4
S31508002860A3FF01F0EBFD064909686431884202D9E5
S3150800287000200149087010BD490100207804002095
S315080028804C0100204801002010B586B004460121FD
S31508002890880300F0ABFF0121480400F087FF0122FE
S315080028A00921C80600F031FB01220A210920C006C9
S315080028B000F02BFB01A801F0C2FE01943021684606
S315080028C0018100214181818101821821C18101A9EB
S315080028D0184801F071FE0121164801F04AFE05A8C4
S315080028E000F069FB01214902684681820121817550
S315080028F01821C17505A90920C00600F0B9FA0121F9
S315080029008902684681824821C17505A90920C00641
S3150800291000F0AEFA1B2168460170032141700121BF
S31508002920817000F00FFF01220221024801F039FEF2
S3150800293006B010BD0038014001B506490098086088
S3150800294002E07E2002F038F9024800680028F8D133
S3150800295008BD000054010020014600220E4B1A61F2
S31508002960CA005A6100229A6105221A6100BF0A4A02
S315080029701069C207D20F002A04D0012212040240AD
S31508002980002AF4D0044A126952085200024B1A610E
S3150800299000229A617047000000E000E010B50021AF
S315080029A00448FFF74BFE022000F04AF801200249CE
S315080029B0087010BD002401408401002000B589B0CC
S315080029C00121084600F0F2FE1A4800F045F801A871
S315080029D000F08EF8184801901848029000216846C1
S315080029E001730420049068460175802141754900E9
S315080029F0C182890001832021817609028183002111
S31508002A00C183018401A90B4800F04CF8012109484B
S31508002A1000F01CF801220221064800F039F80921C5
S31508002A2068460170022141700121817000F08AFE1A
S31508002A3009B000BD0800024000240140BC04002083
S31508002A4001494860704700000000024002685208C9
S31508002A5052000A430260704710B5044620684008D1
S31508002A6040002060002020606060A060E060E1B265
S31508002A70084608380521FEF74DFF01460F20884015
S31508002A800249496808430149486010BD00000240F0
S31508002A90002A03D003680B43036002E003688B43F4
S31508002AA00360704710B50A7A8B7D1A430B7C1A436C
S31508002AB04B7C1A434B8A1A438B8A1A430B8B1A434D
S31508002AC04B8B1A430368094C23401A430260026879
S31508002AD00123DB039A438B8B1A430260CA68426060
S31508002AE00A6882604A68C26010BD00000F80FFFF56
S31508002AF00021016041600172C16001744174418224
S31508002B0081828175018341838183704770B506464A
S31508002B100C4621460A4800F04BF90546002D01D11E
S31508002B20401E70BD0648854202D10648051B00E0D6
S31508002B302D1B224629463046FEF716FF2046F0E7AB
S31508002B4000F4000800FC000870B506460C4621464D
S31508002B500A4800F02DF90546002D01D1401E70BD2A
S31508002B600648854202D10648051B00E02D1B224671
S31508002B7029463046FEF7F8FE2046F0E700F0000842
S31508002B8000F8000870B506460C4621460A4800F0CB
S31508002B900FF90546002D01D1401E70BD0648854235
S31508002BA002D10648051B00E02D1B22462946304661
S31508002BB0FEF7DAFE2046F0E700F8000800000108F4
S31508002BC070B505460C4622460249284600F0B1F87B
S31508002BD0204670BD00F4000870B505460C4622462E
S31508002BE00249284600F0A5F8204670BD00F0000806
S31508002BF010B50446084800690221084306490861D9
S31508002C0008464461006940210843034908610348AE
S31508002C1000F00EF910BD000000200240FF0F000072
S31508002C200C48C068C007C00F002801D001207047B3
S31508002C300848C06804210840002801D00220F6E7A9
S31508002C400448C06810210840002801D00320EEE798
S31508002C500420ECE70020024003480069802108436D
S31508002C6001490861704700000020024030B504465B
S31508002C700D46054800690121084303490861258076
S31508002C800F2000F0D5F830BD0020024010B57E2098
S31508002C9001F092FF064800F00FF87E2001F08CFF45
S31508002CA0044800F009F87E2001F086FF10BD0000F8
S31508002CB000F4000800F0000810B5044600F0ACF86F
S31508002CC02046FFF795FFFFF7C7FF10BD70B503460F
S31508002CD00125002208E050001C5A0748844201D00A
S31508002CE0002506E0501C82B2CE0F76187610964262
S31508002CF0F1DC00BF284670BDFFFF0000F8B50546A9
S31508002D000E46144600F088F87E2001F055FF00278D
S31508002D1007E029883046FFF7A9FFB61CAD1C781CCA
S31508002D2087B2E10F09194910B942F2DCFFF794FF9F
S31508002D30F8BDF8B507460C4615462946204600F064
S31508002D4037F80646002E0DD12046FFF7B5FF0120BD
S31508002D5080022018FFF7B0FF2A4621463846FFF7BB
S31508002D60CDFF24E0012080022018401BB0420AD182
S31508002D70012080022018FFF79FFF2A463146384671
S31508002D80FFF7BCFF13E00120C0022018401BB04229
S31508002D9008D12046FFF790FF2A4631463846FFF706
S31508002DA0ADFF04E02A4631463846FFF7A7FFF8BDCF
S31508002DB0F8B505460E462F46E807C00F002801D08D
S31508002DC000BFFEE731460120C002FEF7B9FD002923
S31508002DD001D000BFFEE700240BE0204670434719E8
S31508002DE031463846FFF772FF012800D108E0601C1B
S31508002DF084B231460120C002FEF7A2FDA042ECDCF7
S31508002E0000BF31460120C002FEF79AFDA04200D15C
S31508002E1000273846F8BD00000248034948600348C1
S31508002E20486070472301674500200240AB89EFCD13
S31508002E3010B5024600BFFFF7F3FE0346521EFF24F5
S31508002E4000E0641E002CFCD1012B01D1002AF2D12E
S31508002E500648006977218843044908613420C86018
S31508002E60002A01D1052010BD1846FCE700200240C3
S31508002E70F8B50246CD782F073F0FCD781026354096
S31508002E80002D01D08D782F431446002011E08506C9
S31508002E902B0E0D88012686403540002D07D0256863
S31508002EA00F269E40B5433E469E4035432560451C49
S31508002EB0E8B20828EBDB141D0D882D1200950020BA
S31508002EC011E085062B0E01258540009E3540002D14
S31508002ED007D025680F269E40B5433E469E4035439B
S31508002EE02560451CE8B20828EBDBCD78282D04D1EF
S31508002EF055690E883543556106E0CD78482D03D1CE
S31508002F0015690E8835431561F8BD70B54D07EB0E8A
S31508002F10082902DA0546203501E0054624352C46FF
S31508002F200F269E402568B54316469E4035432560C4
S31508002F3070BD000038B504460D460920C006844217
S31508002F4003D10121480400F031FC1148844203D121
S31508002F500121000200F02AFC0E48844203D1012117
S31508002F60000200F023FC0C48844203D10121080525
S31508002F7000F01CFC684600F01EF868460580012132
S31508002F8081700021C17069462046FFF771FF38BD80
S31508002F900004004800080048000C004802469068F3
S31508002FA00840002801D0012070470020FCE7416155
S31508002FB07047016170470021C94301800221817071
S31508002FC00421C17070470000F0B58DB000250026B9
S31508002FD000200B900A907E2001F0EEFD00241AE0F6
S31508002FE06100F04A505AFEF754FFEF490590FEF784
S31508002FF075FD0746FEF7C2FF0022EC4B07910690C7
S31508003000FEF75CFE09910890FEF7E0FFA100E84A8A
S315080030105050601C84B2042CE2DBE5498868E54917
S31508003020FEF75CFD0746FEF7A9FFE34AE34B079167
S315080030300690FEF73BFE09910890FEF7C7FF054686
S31508003040DB494868DB49FEF749FD0746FEF796FF68
S31508003050D94ADA4B07910690FEF728FE099108909F
S31508003060FEF7B4FF06462846FEF788FF0022CF4B38
S3150800307003910290FEF71AFE079106902946D0485A
S31508003080FEF7EFFC0746FEF779FF05910490079BCC
S31508003090069AFEF77BFE09910890FEF797FFC94945
S315080030A008603046FEF76AFF0022C04B0391029083
S315080030B0FEF7FCFD079106903146C148FEF7D1FCA4
S315080030C00746FEF75BFF05910490079B069AFEF7F5
S315080030D05DFE09910890FEF779FFBB490860BB4879
S315080030E0008E32282EDABA49488BFEF7EDFEB94A29
S315080030F0B94B01910090FEF7E1FD0022B74B039111
S315080031000290FEF743FE07910690B149488BFEF7F9
S31508003110C0FEB3490290FEF7E1FC0390A948016896
S315080031200398FEF79AFC0746FEF728FF05910490D8
S31508003130079B069AFEF72AFE09910890FEF746FFB6
S315080031400B9028E0A249488BFEF7A3FEA0490790FA
S31508003150888BFEF79EFEA3490590FEF7BFFC0690F6
S315080031600799FEF77EFC07469D49FEF7B7FC984986
S315080031700990488BFEF78DFE99490790FEF7AEFC3D
S315080031800746904801683846FEF767FC0890099993
S31508003190FEF7A4FC0B908D48408E32282EDA8C4917
S315080031A0088BFEF791FE8B4A8B4B01910090FEF738
S315080031B085FD0022894B03910290FEF7E7FD0791F2
S315080031C006908349088BFEF764FE85490290FEF750
S315080031D085FC03907C4801680398FEF73EFC074689
S315080031E0FEF7CCFE05910490079B069AFEF7CEFDE6
S315080031F009910890FEF7EAFE0A9028E07449088BC0
S31508003200FEF747FE72490790C88BFEF742FE7549DE
S315080032100590FEF763FC06900799FEF722FC074621
S315080032206F49FEF75BFC6A490990088BFEF731FE89
S315080032306B490790FEF752FC074663480168384613
S31508003240FEF70BFC08900999FEF748FC0A906648B9
S315080032500B99FEF7ADFB0746FEF75DFE634908606E
S3150800326061480A99FEF7A4FB0746FEF754FE604933
S3150800327008605648008E5D4909684018C003010C6D
S3150800328052480186408E5A4909684018C003010C05
S315080032904E4841864649C8685649FEF7E2FB074646
S315080032A0FEF739FE81B249484030018048487038F7
S315080032B00088FF21F531884272DD002044497039C3
S315080032C008803B490868FEF759FE4B4A4B4B099163
S315080032D00890FEF767FE26D235490868FEF74EFEC7
S315080032E0474A484B09910890FEF75CFE16D24021E2
S315080032F04548FFF753FE002810D13448403040793E
S3150800330001280BD131484030C079002806D1304910
S315080033107039486006212D484030C17101202B497B
S315080033206031887313E0224908683849FEF774FE4D
S315080033300DD226486030807E002804D1002123481B
S315080033406030817303E00121204860308173184999
S3150800335008682F49FEF760FE04D201211B48603039
S31508003360C17303E0002019496031C87317486030FB
S31508003370807B00280FD1154840304079012804D1B8
S3150800338001022148FFF713FE0AE0FF2101311E481A
S31508003390FFF70FFE04E0FF2101311B48FFF709FE86
S315080033A00DB0F0BD7401002000F07F450000084014
S315080033B0E40400200000404125068195438BD43F54
S315080033C0000048438C01002090010020CC03002017
S315080033D07C020020091B9E5E29CB703F00408F406F
S315080033E000007A44002474490000C8419401002072
S315080033F0980100200000C842736891ED7C3FDD3FCC
S315080034009CC420B07268D13F000400486F12233F65
S31508003410333313400148806A70470000C0F7FF1F26
S315080034200148C06A70470000C0F7FF1F01480068DE
S3150800343070470000580100200348006803490978CE
S3150800344040180149086070475801002060010020B3
S3150800345008B50121480400F0A9F90121880400F003
S31508003460A5F96846FFF7A7FD0121C903684601804B
S315080034704821C17069460920C006FFF7F9FC68466D
S31508003480FFF799FD01210903684601804821C170AB
S3150800349069460920C006FFF7EBFC6846FFF78BFD77
S315080034A04021684601800421C17069460148FFF73A
S315080034B0DFFC08BD0004004810B50121C903092036
S315080034C0C006FFF76BFD002869D17748807A002887
S315080034D05AD175484079012837D173482030807E03
S315080034E0002832D171480078401C70490870084697
S315080034F0007805281CDB0020087004216C48FFF7BB
S3150800350058FD694890384089002807D169486A49B2
S315080035104860012164489038418106E000206649E8
S315080035204860002160489038418101F065FB0CE055
S315080035305E480078022808DC5F4840687D2109015A
S31508003540884202D900205C49486057482030807E6E
S31508003550002816D15848406D5849884211D3524818
S3150800356090384089002805D15548534948650020B8
S31508003570486006E04D480078022802DC00204E49E3
S3150800358048600121484881724E48007800280DD1CC
S3150800359001204C49087001214348817106E000204A
S315080035A04849087000214048817181724248C068C4
S315080035B04049884272D900203F49C86000213A48EC
S315080035C081712030807E002862D108213848FFF7B3
S315080035D0F0FC35489038408803285FDA324890383E
S315080035E0408900285AD130484038408E5A280FDA88
S315080035F02D482030C07B00280AD12B484079012865
S315080036004CD129492031887600202B49486045E06D
S3150800361025484079012802D10020274948602248D8
S315080036204038408E5A282ADB27484088274988424E
S3150800363003DC25488088884208DD1B48C0790028B5
S3150800364004D11D49486005211748C1711E484088A4
S315080036500A2803DB1C4880880A2808DA1248C07939
S31508003660002804D11449486004210F48C1710E4846
S31508003670C079002812D102210B48C1710EE00A4810
S315080036802030C07B012809D101210748C17105E016
S315080036900020094948600021034841717E2001F055
S315080036A08BFA0148807910BD0C040020C400002064
S315080036B000040048DC0500000C02002030750000FC
S315080036C0606D0000A201002074010020E60F0000D2
S315080036D008B50121480400F069F80121880400F0C2
S315080036E065F86846FFF767FCFF210E3168460180DA
S315080036F0012181701021C17069461148FFF7B8FB96
S31508003700B62168460180012181701021C170694681
S315080037100920C006FFF7ACFB10210920C006FFF7F9
S3150800372046FC80210920C006FFF741FC0121044818
S31508003730FFF73DFC08210248FFF73BFC08BD0000E7
S31508003740000400488178002925D01749032212026F
S315080037508918027892109200895802789207D30E37
S31508003760FF229A40914342789207120E03789B07EC
S31508003770DB0E9A4011430C4A03231B02D218037826
S315080037809B109B00D1500178CA06D20E01219140A8
S31508003790054A116007E00178CA06D20E0121914058
S315080037A0014A80321160704700E100E0002905D027
S315080037B0054A52690243044B5A6104E0024A5269B7
S315080037C08243014B5A61704700100240002905D018
S315080037D0054AD2690243044BDA6104E0024AD26917
S315080037E08243014BDA61704700100240002905D078
S315080037F0054A92690243044B9A6104E0024A9269B7
S315080038008243014B9A6170470010024010B500F0E0
S3150800381031F804494968F02211400909024A515C05
S31508003820C84010BD001002402201002010B5FFF765
S31508003830EDFF05494968072212021140090A034AA1
S31508003840515CC84010BD0000001002402201002053
S3150800385010B5FFF7DBFF054949680722D202114078
S31508003860C90A034A515CC84010BD00000010024056
S3150800387022010020F8B51E4840680C21084004289B
S3150800388002D008282ED101E01A4C2DE01848403005
S315080038900069C007C00F00280AD0154840300069E3
S315080038A002210840002801D0134802E0114800E030
S315080038B0104807460E4840300069FF2109040840B1
S315080038C0000C451C0A4840300069072109020840D7
S315080038D0000A461C3946694308463146FEF71AF877
S315080038E0044601E0034C00BF00BF2046F8BD0000B7
S315080038F00010024000127A0000093D0070B5044627
S3150800390000250221074800F03AFE002808D005489D
S3150800391000F08EFE20700221024800F028FE0125E4
S31508003920284670BD0038014010B500F001F810BDFA
S3150800393000B585B0624800680121084360490860FF
S3150800394000BF5F480068022108400028F9D05D489A
S315080039505D4908605D480068102108435B490860B6
S3150800396008460068C008C000086057490968481E2C
S315080039705749FDF7CFFF0490544800680499490752
S31508003980490F0843514908604D4840685149084065
S315080039904B494860084640689021084348494860B2
S315080039A0084640684860484800684649884207D93A
S315080039B043484068052109020843414948600BE02D
S315080039C0414800684449884206D93D484068012173
S315080039D0890208433A4948606B4601AA3A48016891
S315080039E03E48FEF7ABFE3648403000698008800046
S315080039F033494031086108460069400840000861BB
S31508003A00684600784007400F0290684600794006ED
S31508003A10400E03902A48C069890508432849C861A9
S31508003A202748403000692E49084025494031086139
S31508003A30039800040299090208432149403109699B
S31508003A4008431F49403108611D48006801210906DD
S31508003A5008431B49086000E000BF194800680121B7
S31508003A60490608400028F7D01548406880088000B5
S31508003A7013494860084640680221084310494860CF
S31508003A8000E000BF0E4840680C2108400828F8D11D
S31508003A900120FEF761FF0A4840681021884308495B
S31508003AA048600120FEF758FF054840688021884392
S31508003AB0034948600120FEF74FFF05B000BD00002E
S31508003AC00010024000A24A043401002000200240EF
S31508003AD000366E010FC0FFFF0051250200127A0062
S31508003AE0FFF800FF042806D1064909690422114394
S31508003AF0044A116105E00349096904229143014A10
S31508003B001161704700E000E010B5FFF795FCA34887
S31508003B100088401CA149088008464068401C486047
S31508003B209F480088401C9E4908809E4800680028D7
S31508003B3004D09C480068401E9A4908609A488079D3
S31508003B40012805D19548C068401C9449C86002E020
S31508003B5000209249C86094482030407D012805D14C
S31508003B608E484069401C8D49486102E000208B4917
S31508003B7048618D48007A012805D18848006C401CA8
S31508003B808649086402E00020844908648349486835
S31508003B900A21FDF7BFFE002927D183482030407A45
S31508003BA081492031097A884207DD7F482030007A2A
S31508003BB0401C7D492031087217E07B482030407A46
S31508003BC079492031097A884200D10EE076482030BA
S31508003BD0407A75492031097A884206DA72482030D7
S31508003BE0007A401E7049203108726F482030807E66
S31508003BF0022804D06C482030807E032804D1674808
S31508003C00806B401C6549886367482030C07A002865
S31508003C100AD165482030807E042805D15F48806C2B
S31508003C20401C5E49886402E000205C4988645E485E
S31508003C302030807E002803D158490865C86426E0EC
S31508003C405948C07A012805D15448006D401C53498B
S31508003C50086502E00020514908655348007B0128A1
S31508003C6012D14E48C06C401C4C49C8644E4820309E
S31508003C70007B002804D108468068401C886006E05E
S31508003C8000204649886002E000204449C864464846
S31508003C90807804280AD14148406D4449884208D2B0
S31508003CA03E48406D401C3D49486502E000203B49BE
S31508003CB04865012109030920C006FFF76FF90028A6
S31508003CC013D039482030807B00280ED136484079F9
S31508003CD001280AD13148806D3549884208D22F48D3
S31508003CE0806D401C2D49886502E000202B498865B7
S31508003CF02D482030007C01280AD12848C06D2D495E
S31508003D00884208D22548C06D401C2449C86502E08F
S31508003D1000202249C86524482030807C012805D126
S31508003D201E48006E401C1D49086602E000201B491B
S31508003D3008661D482030C07C012805D11748406E0A
S31508003D40401C1649486602E00020144948667E2051
S31508003D5000F032FF40211848FFF720F900280AD062
S31508003D600E48C06E1549884208D20C48C06E401CE1
S31508003D700A49C86602E000200849C8660A48203091
S31508003D80007D012805D10548806E401C03498866D8
S31508003D9002E000200149886610BD00000C020020E0
S31508003DA050010020540100200C04002050C30000DC
S31508003DB0881300007017000000040048B888000047
S31508003DC010B51648006801210843144908600846DA
S31508003DD04068134908401149486008460068114977
S31508003DE008400E490860084600680121890488438E
S31508003DF00A49086008464068C321090488430749F8
S31508003E0048600846006808490840044908609F2039
S31508003E1000048860FFF788FD10BD0000001002400E
S31508003E200CC0FFF8FFFFF6FEFFFF8F0008B5012163
S31508003E304804FFF7BBFC022201210920C006FFF750
S31508003E4064F80221684601801821C1700121817039
S31508003E5069460920C006FFF70BF801214804FFF759
S31508003E60A5FC022211460920C006FFF74EF80421D8
S31508003E70684601801821C1700121817069460920B0
S31508003E80C006FEF7F5FF08BD30B587B004460D46F7
S31508003E9001210846FFF79AFC04A800F033F90594B7
S31508003EA068460582002101838176817404A9012070
S31508003EB0800700F0F1F8684600F0D2F860216846FD
S31508003EC001700121417000200190002168460172AD
S31508003ED069460120800700F057F8694601208007E7
S31508003EE000F08AF80821C80600F07EF80821C806FE
S31508003EF000F0B0F84021080600F038F8402108061E
S31508003F0000F03CF80121880700F00AF8012188072B
S31508003F1000F01EF80121880700F00EF807B030BD42
S31508003F20002904D0026880231A43026003E002686D
S31508003F3080239A4302607047002904D0026801234F
S31508003F401A43026003E00268520852000260704792
S31508003F50002905D0426C0123DB031A43426404E0BE
S31508003F60426C0123DB039A43426470478269072344
S31508003F701B039A430B021A4382617047C269702376
S31508003F809A430A43C261704710B5826907231B0327
S31508003F909A430B781B021A4382610A7A12014B78FC
S31508003FA01B011A43036A3024A3431A4302624A6870
S31508003FB082630C4A904213D14A7A12018B781B010C
S31508003FC01A43036AC024A3431A4302624A89920029
S31508003FD08B899B001A4343682401A3431A43426012
S31508003FE010BD0000002C014082690123DB029A43C0
S31508003FF00B021A438261704710B5C26970239A434F
S315080040000B781A43C2610A7A12024B781B021A43CA
S31508004010036A03242402A3431A4302624A68C2635A
S315080040200B4A904213D14A7A12028B781B021A4322
S31508004030036AA400A3431A4302624A8912018B89C0
S315080040401B011A434368A400A3431A43426010BDE8
S31508004050002C0140C26908239A430A43C26170478B
S315080040600021017041708170416001724172418185
S315080040708181704701229207904201D1816301E054
S315080040808AB28263704701229207904201D1C163C6
S3150800409001E08AB2C2637047026803231B029A438F
S315080040A00B891A430260134A904206D001229207EE
S315080040B0904202D0104A904205D1026870239A4372
S315080040C08B781A4302600B4A904205D00B4A9042FD
S315080040D002D00B4A904205D1026B120A12028B7A61
S315080040E01A4302634A68C2620A88826201224261EE
S315080040F070470000002C01400004004000440140C5
S31508004100004801400021C943416000210180018126
S31508004110817081727047000010B50024BD48407D4B
S3150800412000280FD1BC484068BC490968401ABC49F8
S3150800413088420BD90021B748203841710020B5497B
S31508004140887603E0B4484068B4490860B148407CC2
S31508004150002804D001287DD002287CD139E1AD4958
S315080041602039CA8CAC494868E52105F099F8044617
S31508004170A8482038408CA02805DA192201210020F9
S3150800418002F0EEF904E000220121104602F0E8F9F7
S31508004190A0482038C08CE62809D09E482038C08C14
S315080041A0E52804D09B482038C08CE72814D19948C4
S315080041B06038408E9B490988884209D00020954975
S315080041C00875C87408466038408E9649088007E026
S315080041D001209049C87403E000208E490875C87408
S315080041E08D48406E9049884249D98A482038408C83
S315080041F0401E8E490988884239DC86482038408C1A
S31508004200401C8A490988884231DB82482038408C1C
S31508004210CD2834DB7F482038818C408C814203D1FD
S3150800422001207C49087509E000207A4908757A4911
S315080042308866486677482038418C81847648806E3F
S31508004240794988421BD902F0DBFE02F0A5FE01205F
S31508004250704901E01CE0D9E0487400206E494866C0
S31508004260734908706F4908807049088007E06948F3
S315080042702038408C6D490880002067494866002030
S315080042806C49087022460121084602F069F9BEE029
S31508004290604920390A8C60494868B32105F000F85E
S315080042A0044600220121084602F05AF959482038E6
S315080042B0008CB42809D057482038008CB32804D07D
S315080042C054482038008CB5281BD152486038008ED7
S315080042D054490988884210D000204E490875084676
S315080042E02038408C5149088000204A49C87408463D
S315080042F06038008E4B49088007E001204549C8749C
S3150800430003E0002043490875C8744A480078002825
S3150800431010D1414948663F482038408CA02805DD21
S3150800432000220121104602F01BF951E00120414903
S3150800433008704DE03848406E3B49884243D93548B5
S315080043402038408C401E39490988884233DC314878
S315080043502038408C401C3549098888422BDB2D487B
S315080043602038408CA5282BDA2A482038818C408CA6
S31508004370814203D10121274801750AE00021254819
S315080043800175002024498866486622482038418CF1
S3150800439081842148806E2449884211D902201D490A
S315080043A0487402F0C5FE02F0F7FD00201A49486677
S315080043B01F49087004E017482038408C1B490880BC
S315080043C000201549486622460121002002F0C8F857
S315080043D01DE011494868FF21F531FDF79BFA0029D0
S315080043E013D100200C494866134948850122FE214D
S315080043F0572003F0B0FD00220121104602F0B0F864
S3150800440000220121084602F0ABF800E000BF00BF19
S3150800441010BD00002C0400200C0200201001002012
S31508004420C409000016010020DC0500000C0100206C
S31508004430F8000020180100204804002010B5FEF7F7
S31508004440F5FF10BD70B5FFF7E1F905467D21C900F6
S31508004450FDF760FA0446601E0C49884200D90CE054
S31508004460601E0B4948610321081F00F045FC002027
S31508004470074988610720086100BF0420FFF732FB5F
S315080044800021481E00F038FC70BD0000FFFFFF0049
S3150800449000E000E010B50221134800F079F8002882
S315080044A020D0114800F0C4F8C4B21048C0780228D9
S315080044B011D10E480079002810D10D488079AA2814
S315080044C004D10B48C471012108480171AA2C05D1F1
S315080044D00748847102E0204602F05AFF022102488A
S315080044E000F045F810BD0000003801400C0400201B
S315080044F0A405002010B504462146054800F09CF89E
S3150800450000BF0121024800F03AF80028F9D010BD92
S315080045100038014070B505460E4600247E2000F09E
S315080045204BFB00BF20E0042C19DD701EA04216DDEF
S31508004530285D7E2806D17D20FFF7DCFF5E20FFF789
S31508004540D9FF0FE0285D7D2805D1FFF7D3FF5D2051
S31508004550FFF7D0FF06E0285DFFF7CCFF02E0285DF5
S31508004560FFF7C8FF601C84B2B442DCDB70BD416152
S3150800457070478269520852000A43826170470246B0
S3150800458090680840002801D0012070470020FCE709
S315080045900246D0680840002801D001207047002054
S315080045A0FCE7002A03D003690B43036102E00369B1
S315080045B08B4303617047000070B504460D4600261C
S315080045C0E0693021884329790843E061E06944219C
S315080045D08843A9790843E061E06980088000297A60
S315080045E00843E061A0691821884369890843A061E6
S315080045F0A06904218843297B0843A0610B488442AB
S3150800460003D1FFF725F9064602E0FFF70FF906463C
S3150800461030462968FDF77EF9000920623046296888
S31508004620FDF778F90007000F606270BD0038014099
S3150800463001464868C0B27047CAB2026070474B214B
S31508004640C9010160302101710021817101721821AF
S31508004650418100210173704710B51C48408803004A
S3150800466000F03BFB0504111E292A2B001748903041
S315080046700088FF211B31884204DA01211348418052
S3150800468000F0BAFA19E0114890300088FF21053188
S31508004690884204DA02210D48418000F0ADFA0CE0A8
S315080046A00A4890300088F62804DA03210748418032
S315080046B000F0A2FA01E000E000BF00BF0348903016
S315080046C04079002801D100F097FA10BD7C0300203C
S315080046D010B575484088002806D0012845D002281C
S315080046E071D0032840D199E002216F48903081703B
S315080046F040216E48FEF752FC002827D06C494868CE
S31508004700FF21F531FDF706F9C007C00F00280ED1C5
S3150800471080210920C006FEF74CFC01216348FEF7FC
S3150800472048FC10210920C006FEF743FC1CE0802146
S315080047300920C006FEF73BFC01215C48FEF737FC62
S3150800474010210920C006FEF732FC0DE08021092061
S31508004750C006FEF72EFC01215448FEF72AFC10215C
S315080047600920C006FEF725FC9BE001214E48903043
S31508004770817040214D48FEF711FC002813D04C49A2
S315080047804868FF21F531FDF7C5F8C007C00F0028B6
S3150800479004D101214548FEF70CFC08E001214348F5
S315080047A0FEF705FC03E001214048FEF702FC8021E4
S315080047B00920C006FEF7FBFB10210920C006FEF7FC
S315080047C0F6FB6EE0FFE740213848FEF7E7FB0028D6
S315080047D015D037494868FF21F531FDF79BF8C00722
S315080047E0C00F002805D180210920C006FEF7DFFB8F
S315080047F00AE080210920C006FEF7DBFB04E08021E1
S315080048000920C006FEF7D5FB01212848FEF7CFFB95
S3150800481010210920C006FEF7CAFB42E040212348C2
S31508004820FEF7BCFB002815D021494868FF21F53161
S31508004830FDF770F8C007C00F002805D180210920B0
S31508004840C006FEF7B4FB22E080210920C006FEF769
S31508004850B0FB1CE016494868CD21FDF75BF8C00798
S31508004860C00F002805D180210920C006FEF79FFB4E
S315080048700DE00F494868CD21FDF74CF8C007C00F79
S31508004880002804D080210920C006FEF792FB0121EA
S315080048900648FEF78CFB10210920C006FEF787FBA9
S315080048A000BF00BF10BD00007C03002000040048C4
S315080048B00C02002010B5A7488078030000F00DFA16
S315080048C00504447DC0F0EF00A2480088FF21163198
S315080048D0884203DB01219F48817034E09D480088A7
S315080048E0FF210C3188420ADD9A4890384088022810
S315080048F005D0022197489038418000F07DF9402183
S315080049009548FEF74BFB00281DD094494868FF21BF
S31508004910F531FCF7FFFFC007C00F002805D180213D
S315080049200920C006FEF743FB04E080210920C006E3
S31508004930FEF73FFB10210920C006FEF738FB0121D0
S315080049408548FEF734FB03E182480088FF212731BA
S31508004950884203DB02217F4881702DE040217E4892
S31508004960FEF71CFB002827D07C494868FF21F53153
S31508004970FCF7D0FFC007C00F002804D101217648F4
S31508004980FEF715FB03E001217348FEF712FB8021B1
S315080049900920C006FEF70BFB10210920C006FEF70A
S315080049A006FB6C4890384088012805D001216948E3
S315080049B09038418000F020F9CAE066480088FF2157
S315080049C02831884203DB03216248817037E04021A1
S315080049D06148FEF7E3FA002831D060494868FF21AC
S315080049E0F531FCF797FFC007C00F00280ED18021CC
S315080049F00920C006FEF7DDFA01215748FEF7D9FA65
S31508004A0010210920C006FEF7D4FA0DE080210920FE
S31508004A10C006FEF7CCFA10210920C006FEF7C7FA31
S31508004A2001214D48FEF7C3FA4A48903840880028C5
S31508004A3005D0002147489038418000F0DDF887E02E
S31508004A4040214548FEF7AAFA002843D00121090368
S31508004A500920C006FEF7A2FA002807D03F48806D55
S31508004A603F49884202D904213A4881703B4948683F
S31508004A70FF21F531FCF74EFFC007C00F002810D103
S31508004A8080210920C006FEF794FA01213248FEF774
S31508004A9090FA10210920C006FEF78BFA0FE056E0BF
S31508004AA019E080210920C006FEF781FA10210920A5
S31508004AB0C006FEF77CFA01212748FEF778FA254852
S31508004AC090384088002805D0002122489038418037
S31508004AD000F092F83CE040211F48FEF75FFA0028F4
S31508004AE034D01C4890384088002805D00021194841
S31508004AF09038418000F080F81848406D194988427E
S31508004B000ED280210920C006FEF753FA0121124869
S31508004B10FEF74FFA10210920C006FEF74AFA0DE003
S31508004B2080210920C006FEF742FA10210920C00696
S31508004B30FEF73DFA01210848FEF739FA0548203004
S31508004B40807B012802D103210248817000E000BF62
S31508004B5000BF10BD0C040020000400480C02002011
S31508004B609411000030750000034880684008400032
S31508004B700149886070470000002C004080210143ED
S31508004B80014A116070470000002C00400348806805
S31508004B90002801D0012070470020FCE7002C0040C7
S31508004BA010B5FFF7F3FF002804D0FFF7DDFF6620F6
S31508004BB000F002F810BD00004106490E014A1160D6
S31508004BC070470000002C004004494968FF228132E2
S31508004BD091430143014A516070470000002C004090
S31508004BE004494968C909C9014206520E1143014AD6
S31508004BF051607047002C004010B57E20FFF7DCFF9F
S31508004C000948FEF759F8094909480186062130304E
S31508004C1000F03DFA064930318881402202490448AD
S31508004C203030FEF786F810BD00F80008FBAA000031
S31508004C304C03002070B505460C460121C802FEF754
S31508004C40C5FDFF208130FFF7BFFF2046FFF7C8FFED
S31508004C502846FFF793FF70BD0FB410B503A9044BA0
S31508004C60044A029800F09AF810BC08BC04B0184729
S31508004C70DD6F0008040200200FB41CB502460020B0
S31508004C8007AC00290BD0491E01910092064B6A46D3
S31508004C902146069800F082F8009A002111701CBC83
S31508004CA008BC04B018470000795000082021020CFF
S31508004CB001D010211046020A01D01046083902090F
S31508004CC001D01046091F820801D01046891E4208E5
S31508004CD001D0881E7047081A704730B47446641E9F
S31508004CE02578641CAB4204D3635D5B00E31830BCD3
S31508004CF018471D46F8E7000010B5002819DB1A4AC0
S31508004D0003231B02D21883089B00D2588307DC0EA4
S31508004D10FF23A3409A438B071B0E8407E40EA34088
S31508004D201A43114B032424021B198408A4001A51A0
S31508004D3018E00E4A03071B0F083B9B089B00D25836
S31508004D408307DC0EFF23A3409A438B071B0E8407B9
S31508004D50E40EA3401A43054B0407240F083CA40895
S31508004D60A4001A5110BD000000E100E01CED00E0AF
S31508004D7002E008C8121F08C1002AFAD17047704716
S31508004D80002001E001C1121F002AFBD17047000074
S31508004D90014908607047000008020020FFB58FB07F
S31508004DA00F460446002606E025280AD0129A1199CD
S31508004DB09047641C761C20780028F5D1304613B03D
S31508004DC0F0BD00250121A14A009500E00543641CB9
S31508004DD023780846203B98401042F7D120782E28A1
S31508004DE015D1042005436078641C2A280AD101CF0E
S31508004DF0641C00900BE000990A2251433039401890
S31508004E00641C00902078014630390929F3D92078A6
S31508004E106C280ED004DC4C2813D06A2812D104E082
S31508004E2074280ED07A280DD10BE0012040050543E1
S31508004E3007E00121090562780D43824201D16D1808
S31508004E40641C641C2078864669284AD008DC002839
S31508004E50B4D058286DD0632810D0642808D140E013
S31508004E6070286BD0732812D0752860D0782860D047
S31508004E70129A704611999047761CE5E0387869468B
S31508004E8008720020487202A80190012003E03868E1
S31508004E9001900020C0433F1D69070CD5002500E09E
S31508004EA06D1C00998D420FDA8542F9DB0199495D3F
S31508004EB00029F5D108E0002500E06D1C8542FCDBE1
S31508004EC00199495D0029F8D1761907E001980199F9
S31508004ED00078491C0191129A119990476D1EF5D2D6
S31508004EE0B2E00A20029000216802400F03910228CE
S31508004EF00CD001CFC117844600290DDA6246084650
S31508004F0052420021814194462D2008E0FF1DFF08EA
S31508004F10FF0003CF8446EFE7280504D52B206A4611
S31508004F20107401203CE0E8073AD02020F7E70A2071
S31508004F3000E0102000210391029007E01020029063
S31508004F400021042005430820039100906802400FC1
S31508004F50022810D001CF0021844600200D90280792
S31508004F601FD5704670280CD0029A1020039B424029
S31508004F701A430CD015E0FF1DFF08FF0003CF844637
S31508004F80EBE740206A46107401200D900CE060465D
S31508004F90084306D030206A461074704650740220C2
S31508004FA00D907046582804D029A001900DA80E909F
S31508004FB00DE02CA0F9E76046039B029AFDF736F848
S31508004FC0019B84469B5C0E9A521E0E921370604695
S31508004FD00843F0D10E9805A9081A203001906807F1
S31508004FE001D5009801E0012000900199884203DD6F
S31508004FF001460198081A00E000200025009006E006
S3150800500004A8129A405D119990476D1C761C0D985C
S315080050108542F5DB04E0129A302011999047761CF8
S315080050200099481E00900029F5DC08E00E980E99B4
S315080050300078491C0E91129A11999047761C01998D
S31508005040481E01900029F1DC641CB4E60928010019
S3150800505030313233343536373839616263646566E0
S3150800506000000000303132333435363738394142A2
S3150800507043444546000000004A68002A06D00A68EC
S31508005080531C0B6010704868401E4860704710B586
S3150800509002460023002901D1002010BD03E0148830
S315080050A0921CE01883B208464C1EA1B20028F6D11D
S315080050B01846F2E710B5BE484079002864D1102199
S315080050C00920C006FDF773FF80210920C006FDF7F9
S315080050D06EFF0121B748FDF76AFF0020B449203169
S315080050E08876002301221946184603F069F9002339
S315080050F01A461946184603F063F9AF484068FF2177
S31508005100F531884204D20421AA48FDF752FF4DE141
S315080051100421A848FDF74BFFA7484068A7498842DD
S31508005120F5D9A348807A002817D1A34840687D217D
S315080051304901884201D2FFF78FFA08219D48FDF7F9
S3150800514036FF00219A48C171002099492031C8725A
S3150800515008739949486248630CE040219548FDF771
S315080051601DFF002806D000219148203081760121B4
S315080051702038417120210920C006FDF718FF7D203F
S3150800518040018D49486011E189482030807E03003E
S31508005190FFF7A3FD060470B3FEFDFC6F00208449EB
S315080051A02031C87208738449486248630023012283
S315080051B01946184603F004F900231A4619461846F4
S315080051C003F0FEF87A484038418E01874030C078AF
S315080051D0012808D1784840697949884202D90021CE
S315080051E07348C17010BD744840687D210901884222
S315080051F027D90020734908706D48807A002802D1A3
S315080052006D49486002E070486B494860402169482A
S31508005210FDF7C4FE00280CD1FFF71EFA08216548E1
S31508005220FDF7C5FE7E20FFF7C7FC1E20FDF784FBB1
S3150800523002E000206049486004215E48FDF7B7FE99
S3150800524017E020210920C006FDF7B3FE08215948BA
S31508005250FDF7AFFE58484068FF21F531884208D966
S31508005260534890384089002803D104215148FDF756
S315080052709EFE9AE050484068FF21F531884204D2E4
S3150800528004214C48FDF795FE03E004214948FDF743
S315080052908EFE4748C078052817D100220121084606
S315080052A001F05EF942484038018E4030C08B814299
S315080052B005DA64220121002001F052F907E00022F4
S315080052C00121104601F04CF901E0FEF725FF3848A8
S315080052D04038418E4030C08B81420DDB344840381F
S315080052E0018E4030C08B814206DB0020324948607F
S315080052F002202F492031887657E02F484068FF2141
S31508005300F531884204D204212A48FDF752FE03E00B
S3150800531004212848FDF74BFE274840682B49884258
S315080053201ED92348C08BD2281AD12148C08CCF2831
S3150800533012DB1F48C08CD5280EDA01201C49203103
S3150800534088741D48006E1E49884209D90122FE212B
S31508005350672002F000FE03E000201549203188741A
S315080053601348C07805281AD100220121084601F001
S31508005370F7F80F484038018E4030C08B814208DA72
S315080053803C220121002001F0EBF80AE00CE00AE0DB
S3150800539008E000220121104601F0E2F801E0FEF7DC
S315080053A0BBFE02E001E000E000BF00BF00BF19E756
S315080053B00C040020000400480C020020B80B000072
S315080053C088130000C4000020C4090000102700004C
S315080053D010B5BD484079002864D110210920C006BF
S315080053E0FDF7E5FD80210920C006FDF7E0FD012156
S315080053F0B648FDF7DCFD0020B34920318876002346
S3150800540001221946184602F0DBFF00231A46194600
S31508005410184602F0D5FFAE484068FF21F5318842AC
S3150800542004D20421A948FDF7C4FD4AE10421A7488E
S31508005430FDF7BDFDA6484068A6498842F5D9A248A9
S31508005440807A002817D1A24840687D214901884200
S3150800545001D2FFF701F908219C48FDF7A8FD0021B4
S315080054609948C171002098492031C8720873984933
S31508005470486248630CE040219448FDF78FFD0028F8
S3150800548006D0002090492031887601218E48417146
S3150800549020210920C006FDF78AFD7D2040018C49A0
S315080054A048600EE188482030807E0300FFF715FC2F
S315080054B0060474B0FBFAF973002083492031C872D8
S315080054C000218148203001730020814948624863E1
S315080054D0002301221946184602F072FF00231A46D5
S315080054E01946184602F06CFF77484038418E018706
S315080054F04030C078012808D1754840697649884205
S3150800550002D900217048C17010BD714840687D21DC
S315080055100901884227D90020704908706A48807AAC
S31508005520002802D16A49486002E06D486849486027
S3150800553040216648FDF732FD00280CD1FFF78CF8AC
S3150800554008216248FDF733FD7E20FFF735FB1E2054
S31508005550FDF7F2F902E000205D49486004215B4846
S31508005560FDF725FD17E020210920C006FDF721FDDE
S3150800557008215648FDF71DFD55484068FF21F531BD
S31508005580884208D9504890384089002803D1042118
S315080055904E48FDF70CFD93E04D484068FF21F53174
S315080055A0884204D204214948FDF703FD03E004219B
S315080055B04648FDF7FCFC4448C078062817D1002267
S315080055C00121104600F0CCFF3F484038418E40305C
S315080055D0C08B814205DA50220121084600F0C0FF3F
S315080055E007E000220121084600F0BAFF01E003F0B7
S315080055F0A9FD35484038418E4030C08B814206DBD4
S3150800560000203349486002202F492031887657E028
S315080056102F484068FF21F531884204D204212B48DF
S31508005620FDF7C7FC03E004212848FDF7C0FC28481D
S3150800563040682C4988421ED92348C08BD2281AD1E3
S315080056402148C08CCF2812DB1F48C08CD5280EDA1B
S3150800565001201D49203188741D48006E1E49884264
S3150800566009D90122FE21672002F075FC03E000201B
S315080056701549203188741448C07806281AD10022A2
S315080056800121104600F06CFF0F484038418E40302B
S31508005690C08B814208DA3C220121084600F060FFEF
S315080056A00AE00CE00AE008E000220121084600F0C2
S315080056B057FF01E003F046FD02E001E000E000BF0D
S315080056C000BF00BF20E700000C04002000040048CB
S315080056D00C020020B80B000088130000C40000204C
S315080056E0C40900001027000010B56D48407900284D
S315080056F064D110210920C006FDF759FC8021092034
S31508005700C006FDF754FC01216648FDF750FC002150
S31508005710634820308176002301221946184602F094
S315080057204FFE00231A461946184602F049FE5E48FF
S315080057304068FF21F531884204D204215948FDF713
S3150800574038FCABE004215748FDF731FC5648406861
S3150800575056498842F5D95248807A002817D15248C6
S3150800576040687D214901884201D2FEF775FF08216C
S315080057704C48FDF71CFC00214948C17100204849E6
S315080057802031C87208734849486248630CE04021D2
S315080057904448FDF703FC002806D000214048203085
S315080057A0817601212038417120210920C006FDF7A4
S315080057B0FEFB7D2040013C4948606FE038482030B8
S315080057C0807E002804D0012865D0022865D163E0D0
S315080057D0002133482030C172002031492031087336
S315080057E03149486248632E484038418E0187403027
S315080057F0C078012808D12C4840692D49884202D929
S3150800580000212748C17010BD274840687D2109013D
S31508005810884227D90020274908702148807A00281D
S3150800582002D12149486002E023481F4948604021C7
S315080058301C48FDF7B3FB00280CD1FEF70DFF082125
S315080058401848FDF7B4FB7E20FFF7B6F91E20FDF7D2
S3150800585073F802E000201449486004211148FDF756
S31508005860A6FB17E020210920C006FDF7A2FB0821A8
S315080058700C48FDF79EFB0C484068FF21F53188422D
S3150800588008D9074890384089002803D104210548DB
S31508005890FDF78DFB01E000E000BF00BF00BFB2E7E7
S315080058A00C040020000400480C020020B80B00007D
S315080058B088130000C4000020C4090000F0B587B0B2
S315080058C00020069005900024002504900026002755
S315080058D0F748407D012814D1F64840694B21C90094
S315080058E088420ED90020F2494875F2494861F249C2
S315080058F00880F2490870FF210131EF48801DFCF746
S315080059004CF8EB482038007901286CD17E20FFF747
S3150800591053F9E948C0790002E749097A084306902D
S31508005920E548407A0590E448847AC67A0246117BAF
S31508005930507B01F081FE0746DF4AD17A107B01F0E1
S315080059407BFE05460021DA48203801710121203006
S3150800595041750020D7494861D94A0698811A90426C
S3150800596042D03CDCD74A811A90423ED01EDCD64A49
S31508005970811A90423AD010DCD44A811A904236D025
S3150800598006DC442861D0D2494018002871D19CE22F
S3150800599001296FD00229F9D1D1E201296BD0022958
S315080059A06AD0032969D01029F0D151E32A297DD07C
S315080059B00CDC22297BD004DC012979D01129E5D118
S315080059C0FAE3232975D02929E0D15DE0312971D080
S315080059D0332970D044296FD05729D7D19CE0881E27
S315080059E0282846D204E0F2E376E092E3C1E27AE2BE
S315080059F043007B449B885B009F446A0066007200F4
S31508005A003B003B003B003B003B003B003B003B00B0
S31508005A103B003B003B003B003B003B0021020D02E4
S31508005A204F022B0274018501D5013B003B003B0068
S31508005A304000300148019C01BA013B003B009F0031
S31508005A40AB00F7001101C500DF000598062809D14B
S31508005A50A048007800280BD102F0A8FA01209D4939
S31508005A60087005E00598062802DD012002F09EFA76
S31508005A7012E2FDE34BE288E29CE2C6E20022FE2146
S31508005A80E82002F068FAF3E78949203909880A22EA
S31508005A9051430846FCF7F2F98F490090FCF71EF8C7
S31508005AA08E490190FBF7DDFF029006E0C7E39AE313
S31508005AB07CE3AEE318E0E1E3EFE3FCF72CFA80B20F
S31508005AC0039002F01CFAD3E7032002F06FFACFE73F
S31508005AD0042002F06BFACBE7052002F067FAC7E765
S31508005AE0022002F063FAC3E7012C0AD1714870302C
S31508005AF0008B0123002297210090FE2002F0CBF9AB
S31508005B0009E06C487030408B0223002297210090F0
S31508005B10FE2002F0C0F9FAE304217148FDF749FABC
S31508005B20C820FCF709FF04216D48FDF740FA00225A
S31508005B30FE21BD2002F00FFAE9E35D48807E0028C9
S31508005B4006D05B486038028E418E002002F034F998
S31508005B50DDE3002C0AD156486038408E00231A46E9
S31508005B60F0210090FE2002F096F90BE0012C09D1F5
S31508005B704F486038008E01230022F0210090FE2055
S31508005B8002F089F9C3E3002C0AD14A4870304088EC
S31508005B9000231A46F3210090FE2002F07CF90BE060
S31508005BA0012C09D143487030808901230022F32152
S31508005BB00090FE2002F06FF9A9E3002C03D13D48BE
S31508005BC07030458002E03B48703085813948703036
S31508005BD08089FF21F531884206DA01F0DDF90022D5
S31508005BE0FE21F42002F0B7F991E3002C0AD13148DE
S31508005BF07030808800231A46F1210090FE2002F0BA
S31508005C004AF90BE0012C09D12A487030C0890123D2
S31508005C100022F1210090FE2002F03DF977E3002CE6
S31508005C2003D124487030858004E0012C02D1214834
S31508005C307030C5811F4870308088FF21F531884251
S31508005C400BDC1C487030C089884206DC01F0A4F9D8
S31508005C500022FE21F22002F07EF958E3002C0AD138
S31508005C6014487030C08800231A46E9210090FE20A7
S31508005C7002F011F909E0012C07D1192001230022AD
S31508005C80E9210090FE2002F006F940E3002C02D13B
S31508005C9008487030C580FF202D30854206DA01F0AD
S31508005CA07BF90022FE21EA2002F055F92FE30000D5
S31508005CB02C0400200C020020A4050020F10100207D
S31508005CC0CBFE000066FE000055FE000052FE0000F6
S31508005CD0AF01FFFF000200200000A0400000E040E6
S31508005CE000040048002C0CD1FE4800896421484372
S31508005CF080B200231A46E2210090FE2002F0CBF87B
S31508005D0000E000BF03E3002C06D164212846FBF718
S31508005D1017FE81B2F3480181F2480089FF21F53167
S31508005D20884206DC01F038F90022FE21E32002F061
S31508005D3012F9ECE2002C0CD1EA4840896421484368
S31508005D4080B200231A46EB210090FE2002F0A3F849
S31508005D500DE0012C0BD1E348008A6421484380B248
S31508005D6001230022EB210090FE2002F094F8CEE2F7
S31508005D70002C07D164212846FBF7E2FD81B2D948F9
S31508005D80418108E0012C06D164212846FBF7D8FD9D
S31508005D9081B2D448018201F0FFF80022FE21EC20EE
S31508005DA002F0D9F8B3E2012C19D1CF48408803286C
S31508005DB00BDACD484089002807D10121CA48B030FE
S31508005DC081760020C749703948600022FE21E42008
S31508005DD002F0C1F80121C448903041711AE0002C44
S31508005DE013D10021C048903041710020BE49B0311E
S31508005DF088760022FE21E42002F0ADF80020BB4997
S31508005E000870B8497039486004E00022FE21E42091
S31508005E1002F0A1F87BE2002C0FD1B548C07A3228EF
S31508005E200CDCB348C17AAF48418201F0B5F80022CC
S31508005E30FE21DF2002F08FF800E000BF67E2A948E4
S31508005E40408A00231A46DE210090FE2002F023F83D
S31508005E505DE2002C0FD1A648C07A32281CDCA44883
S31508005E60C17AA048818201F097F80022FE21E1203C
S31508005E7002F071F810E0012C0ED19D48C07A322844
S31508005E800ADC9B48C17A9748C18201F085F800224E
S31508005E90FE21E12002F05FF839E2002C09D1914891
S31508005EA0808A00231A46E0210090FE2001F0F3FFC5
S31508005EB00AE0012C08D18B48C08A01230022E02180
S31508005EC00090FE2001F0E7FF21E28A498548818398
S31508005ED0C1830184418401F05FF80022FE2151202C
S31508005EE002F039F813E2002C10D1002E03D17E48B7
S31508005EF0903007840AE0012E03D17B48903047840E
S31508005F0004E0022E02D178489030C784FFE1002CC5
S31508005F1014D1FDF77FFA04900498000C00231A4662
S31508005F2053210090FE2001F0B6FF049880B20123A9
S31508005F30002253210090FE2001F0ADFFE7E1002C7E
S31508005F400AD16848C08B00906648838B002254218A
S31508005F50FE2001F066FF0BE0012C09D16148408C58
S31508005F6000906048038C01225421FE2001F059FF5D
S31508005F70CDE1002C08D101215B489030C170002288
S31508005F8002215D48FEF70DFBC1E1002C11D1FF216E
S31508005F9001315748801DFBF700FD00205449088051
S31508005FA0022151489030C1700022FE21562001F08E
S31508005FB0D2FFACE1002C18D100214B48B030417417
S31508005FC000204B490880032147489030C1700121C1
S31508005FD0417120308176002042497039486000229C
S31508005FE0FE21572001F0B7FF0EE0012C0CD100214D
S31508005FF03D489030C17000203B49B0318876012277
S31508006000FE21572001F0A7FF81E1002C17D10020BF
S315080060103549B031487436490880042132489030F1
S31508006020C170012141712030817600202D497039D7
S3150800603048600022FE21582001F08DFF07E0012C60
S3150800604005D1002128489030C170203081765EE164
S31508006050002C1AD1002026490880062122489030B3
S31508006060C1700121417101201F49B0318876002095
S315080060701C4970394860B4211B489030C1830022FE
S31508006080FE21652001F067FF42E0012C18D10020AF
S3150800609017490880062114489030C17001214171C2
S315080060A02030817600200F4970394860D2210E4889
S315080060B09030C1830022FE21652001F04CFF27E0C5
S315080060C0022C25D100200A4908800621064890306E
S315080060D0C1700121417101200349B0318876002041
S315080060E000490BE07C0200207C030020000200200F
S315080060F0A4050020041000000038014070394860EB
S31508006100F0218448C1830022FE21652001F023FF87
S31508006110FDE0002C17D100207F49088005217D4825
S31508006120C1700121417101207A4920318876002009
S315080061307A494860B4217748C1830022FE21662047
S3150800614001F009FF30E0012C17D1002072490880C0
S3150800615005217048C1700121417101206D49203126
S31508006160887600206D494860D2216A48C18300229A
S31508006170FE21662001F0EFFE16E0022C14D1002065
S315080061806549088005216348C170012141712030A5
S315080061908176002061494860F0215E48C18300226B
S315080061A0FE21662001F0D7FEB1E005E0002159483E
S315080061B0C17020308176AAE0002C09D10721554804
S315080061C0C1700022FE21772001F0C5FE0AE09FE09B
S315080061D0012C07D100214F48C1700122FE217720EA
S315080061E001F0B9FE93E0002C12D1642201210020AF
S315080061F000F0B6F900220121084600F0B1F90120A5
S315080062004449203188760022FE21882001F0A3FE29
S315080062107DE0002C12D164220121084600F0A0F985
S3150800622000220121104600F09BF90120394920314E
S3150800623088760022FE21892001F08DFE67E0384924
S3150800624038480068FBF70DFC0190FBF764FE80B246
S315080062503349039034480068FBF703FC0190FBF7C9
S315080062605AFE80B20290039800900022902100E026
S315080062704CE0FE20029B01F0D4FD48E0002C33D10F
S31508006280002E0BD125487030C7830022FE215220EC
S3150800629001F061FE00F080FE26E026E0012E0AD11C
S315080062A01E487030878300F077FE0122FE215220B7
S315080062B001F051FE18E0022E0AD1184870304784C2
S315080062C000F06AFE0222FE21522001F044FE0BE095
S315080062D0032E09D111487030078400F05DFE0322B1
S315080062E0FE21522001F037FE11E0002C0DD10120CD
S315080062F0084920318876012106484171012005495F
S315080063002031887500200549486000E000BF00BFBD
S3150800631007B0F0BD0C040020A40500200C020020E4
S3150800632000007A44900100208C010020F0B589B065
S3150800633000200890079006905048007901287DD1E2
S315080063404F488079AA287AD14D48C079322877DA19
S315080063504B48C079002873DD4949C9790846193878
S31508006360FBF78CFD08900898FBF708FE0646454A99
S31508006370454BFBF7A3FC04460022444BFBF7ECFB1A
S315080063800391029042480068FBF7F8FD01910090DE
S31508006390039B029AFBF7FAFC05910490FBF716FE9D
S315080063A007900898FBF7EAFD0446364A364BFBF792
S315080063B085FC0022354B01910090FBF7CDFB03913C
S315080063C0029034480068FBF7D9FD0646039B029AFB
S315080063D0FBF7DCFC05910490FBF7F8FD06902E49C7
S315080063E00798FBF70FFE38D22C490798FBF714FEDF
S315080063F033D229490698FBF705FE2ED22749069877
S31508006400FBF70AFE29D226490798FBF72AFB04461A
S31508006410FBF781FD81B22348418321490698FBF7A2
S3150800642020FB0446FBF777FD81B21E48018300F086
S31508006430B3FD1C48408B00901A4802E01BE017E0A9
S3150800644013E0038B00226021FE2001F0EAFC012202
S31508006450FE21562001F07FFD04E00222FE2156208F
S3150800646001F079FD00210548C17000210348C1707B
S3150800647000210248017109B0F0BD00000C0400209B
S31508006480A4050020091B9E5E29CB703F0000F03F43
S315080064908C01002090010020000018410000E04017
S315080064A000007A447C02002029494A88498A511A00
S315080064B0814209DB264970398968254A703AD162D2
S315080064C00021244A11701AE021494988814216DCC4
S315080064D020490978002912D11F490A880A8301210F
S315080064E01C4A11701A4970398968194A703AD26A71
S315080064F0891A174A703A51621146896851631449D4
S315080065008A88898A511A814209DB0021134A117047
S315080065100F49703989680E4A703A116317E00C49B9
S315080065208988814213DC0D49097800290FD10A4967
S315080065300A884A830121094A117005497039896810
S31508006540034A703A126B891A014A703A9162704787
S315080065507C020020E40000200C040020E500002056
S3150800656070B505460E461446002E02D0012E4AD1B5
S3150800657020E0002D02D0012D1AD10CE06021012067
S315080065808007FDF7F3FC002101208007FDF772FD67
S315080065901E4804700CE0602101208007FDF7EEFC20
S315080065A0002101208007FDF76EFD1948047000BF21
S315080065B000BF28E0002D02D0012D22D110E013489B
S315080065C00078A0420BD0602101208007FDF7CEFCA1
S315080065D0214601208007FDF74DFD0C48047010E0A8
S315080065E00B480078A0420BD0602101208007FDF7F8
S315080065F0C5FC214601208007FDF745FD04480470C7
S3150800660000BF00BF00BF00BF70BD0000A30100208F
S31508006610A401002010B5F3484079012879D1F14842
S315080066202030007E0028F9D1EE48C0790300FEF735
S3150800663054FB0805075DB0FDFCFBFAF9002010BD08
S31508006640E9494868FF219131FBF764F98007800F13
S31508006650002809D180210920C006FCF7A8FC0121E1
S31508006660E248FCF7A4FC3AE0DF494868FF2191318B
S31508006670FBF750F98007800F012809D180210920EE
S31508006680C006FCF796FC0121D848FCF790FC26E0EA
S31508006690D5494868FF219131FBF73CF98007800FFF
S315080066A0022809D180210920C006FCF780FC0121B7
S315080066B0CE48FCF77CFC12E0CB494868FF219131B3
S315080066C0FBF728F98007800F032808D10121C7485E
S315080066D0FCF76FFC80210920C006FCF768FC102136
S315080066E00920C006FCF763FC0120A8E7BE494868F4
S315080066F0C821FBF70FF98007800F00280AD18021EF
S315080067000920C006FCF753FC0121B848FCF74FFCEA
S3150800671038E065E1B4494868C821FBF7FBF880070B
S31508006720800F012809D180210920C006FCF741FC09
S315080067300121AE48FCF73BFC24E0AB494868C82178
S31508006740FBF7E8F88007800F022809D18021092085
S31508006750C006FCF72CFC0121A448FCF728FC11E034
S31508006760A1494868C821FBF7D5F88007800F032898
S3150800677008D101219D48FCF71CFC80210920C00690
S31508006780FCF715FC10210920C006FCF710FC0120B7
S3150800679055E795494868C821FBF7BCF88007800F7C
S315080067A0002809D180210920C006FCF700FC012138
S315080067B08E48FCF7FCFB3DE08B494868C821FBF78F
S315080067C0A9F88007800F012809D180210920C00671
S315080067D0FCF7EFFB01218548FCF7E9FB2AE0824933
S315080067E04868C821FBF796F88007800F022809D168
S315080067F080210920C006FCF7DAFB01217B48FCF75B
S31508006800D6FB17E078494868C821FBF783F8800764
S31508006810800F03280ED101217448FCF7CAFB80219A
S31508006820092004E0DBE0B2E05FE034E009E0C006FE
S31508006830FCF7BDFB10210920C006FCF7B8FB0120B8
S31508006840FDE669494868FF212D31FBF763F8C00763
S31508006850C00F002805D180210920C006FCF7A7FB38
S315080068600EE061494868FF212D31FBF753F8C00750
S31508006870C00F002804D080210920C006FCF799FB28
S3150800688010210920C006FCF792FB01215748FCF7A6
S315080068908EFB0120D3E654494868FF219131FBF766
S315080068A039F8C007C00F002805D180210920C00685
S315080068B0FCF77DFB0EE04C494868FF219131FBF758
S315080068C029F8C007C00F002804D080210920C00677
S315080068D0FCF76FFB10210920C006FCF768FB0121B5
S315080068E04248FCF764FB0120A9E63F494868C821ED
S315080068F0FBF710F88007800F002809D180210920AE
S31508006900C006FCF754FB01213848FCF750FB37E07A
S3150800691035494868C821FAF7FDFF8007800F012826
S3150800692009D180210920C006FCF743FB01212F4825
S31508006930FCF73DFB24E02C494868C821FAF7EAFF32
S315080069408007800F022809D180210920C006FCF79C
S315080069502EFB01212548FCF72AFB11E0224948684D
S31508006960C821FAF7D7FF8007800F032808D101212D
S315080069701E48FCF71EFB80210920C006FCF717FB02
S3150800698010210920C006FCF712FB012057E616491C
S315080069904868C821FAF7BEFFC007C00F002805D10E
S315080069A080210920C006FCF702FB0DE00E49486865
S315080069B0C821FAF7AFFFC007C00F002804D080210E
S315080069C00920C006FCF7F5FA10210920C006FCF7D5
S315080069D0EEFA01210548FCF7EAFA01202FE600BF86
S315080069E000BF2CE60C0400200C020020000400481E
S315080069F010B5FE48807E002874D0FC486038408E6A
S31508006A00FF217D31884204DCF8486038008E8842D0
S31508006A101CDDF6482038C079002817D1F44840888C
S31508006A200A2813DDF2484088F24988420EDAF0480F
S31508006A3080880A280ADDEE488088884206DA00201F
S31508006A40ED4948600321E9482038C171EA48006CDD
S31508006A50EA4988420AD9E5482038C079002805D18C
S31508006A60E54948600321E1482038C171DF48807E46
S31508006A70042838D1DD48C07A00282BD1DB482038D5
S31508006A80C07A01281ED1DC48006DDD49884231D91B
S31508006A900020D9490865D5486038C18E008E8142E4
S31508006AA00BDBD2482038C079002823D1D249486068
S31508006AB00721CE482038C1711CE0CC486038018EC9
S31508006AC0C18617E00020CC490865C8486038018EA1
S31508006AD0C1860FE00020C8490865C4486038018EA1
S31508006AE0C18607E028E00020C3490865BF4860382A
S31508006AF0018EC186BD48807E01282BD1BB4820382F
S31508006B00007B01281ED1BC48C06CBD49884228D9E3
S31508006B100020B949C864B5486038818E408E8142E4
S31508006B200BDBB2482038C07900281AD1B249486030
S31508006B300721AE482038C17113E0AC486038418E51
S31508006B4081860EE00020AC49C864A8486038418EAA
S31508006B50818606E00020A849C864A4486038418EAA
S31508006B608186A24820384079012877D19F48203865
S31508006B70C07900280BD0002301221946184601F0D7
S31508006B801FFC00231A461946184601F019FC9748B7
S31508006B902038C0790300FEF7A0F80805073C71A461
S31508006BA0D8FDFCFB002010BD93484068E121C900D0
S31508006BB0884229D910210920C006FCF7F8F9802156
S31508006BC00920C006FCF7F3F901218E48FCF7EFF916
S31508006BD00120864908760846807D002807D186491F
S31508006BE048600021814820384171C17108E0824817
S31508006BF04068AF210901884202D900207E494860D1
S31508006C0001207A49C87502E00020784908760120F3
S31508006C10C9E7794840687C4988422AD91021092061
S31508006C20C006FCF7C4F980210920C006FCF7BFF9A5
S31508006C3001217448FCF7BBF901206C49087608461F
S31508006C40807D00280BD16C494860002167482038B0
S31508006C504171C1710020684948600DE02BE1664822
S31508006C604068AF210901884206D900206249486078
S31508006C7002E000205D490876012094E75E484068F6
S31508006C806249884228D910210920C006FCF78FF9E5
S31508006C9080210920C006FCF78AF901215948FCF72A
S31508006CA086F90120514908760846807D00280AD1D0
S31508006CB05149486000214D4820384171C171002072
S31508006CC04D4948600BE04C4840685149884206D90E
S31508006CD000204949486002E000204449087601201E
S31508006CE061E7454840687D210901884228D9102175
S31508006CF00920C006FCF75BF980210920C006FCF7CD
S31508006D0056F901213F48FCF752F901203749087620
S31508006D100846807D00280AD1374948600021334853
S31508006D2020384171C1710020334948600BE0324870
S31508006D3040683349884206D900202F49486002E056
S31508006D4000202A49087601202DE72B484068E121D2
S31508006D50C90088422DD910210920C006FCF727F959
S31508006D6080210920C006FCF722F901212548FCF7F5
S31508006D701EF901201D4908760846807D00280ED197
S31508006D801D4948600021194820384171C17102E047
S31508006D9090E05CE012E00020174948600CE01648D5
S31508006DA04068AF210901884206D900201249486087
S31508006DB002E000200D4908760120F4E60E484068F6
S31508006DC01349C83988423CD910210920C006FCF766
S31508006DD0EEF880210920C006FCF7E9F801210948E8
S31508006DE0FCF7E5F801200149087613E02C04002099
S31508006DF074010020E60F00000C020020701101004B
S31508006E00B80B000000040048A4060000C4090000EE
S31508006E10AC0D00000846807D002809D12749486046
S31508006E20002127484171C1710020244948600CE0BF
S31508006E30224840682349884207D900201F494860EC
S31508006E4003E000211E48203001760120ABE61B48EE
S31508006E5040681D49884227D910210920C006FCF739
S31508006E60A6F880210920C006FCF7A1F801211748D9
S31508006E70FCF79DF80121124820300176807D002814
S31508006E8009D10E49486000210D484171C1710020A1
S31508006E900A4948600CE0094840680D49884207D904
S31508006EA000200649486003E000200549203108769D
S31508006EB0012078E600BF00BF75E600000C0200203E
S31508006EC00C040020CC100000A406000000040048B2
S31508006ED08C0A000010B5052421E080212C48FAF719
S31508006EE05CFD80212A48FBF711FE12212848FEF78F
S31508006EF0CEF82749898C88420CD125483038008E2F
S31508006F002449884204D000F051FC00F045F800E01E
S31508006F1010BD04E0002000E0401C8028FCDB204671
S31508006F20611ECCB20028D8D100BF052423E08021F9
S31508006F301748FAF732FD80211548FBF705FE12219E
S31508006F401348FEF7A4F81249898C88420ED11048D6
S31508006F503038008E0F49884204D000F027FC00F034
S31508006F601BF802E000F018F8D2E704E0002000E081
S31508006F70401C8028FCDB2046611ECCB20028D6D1F6
S31508006F8000BF00F013FC00F007F800BFC0E70000E0
S31508006F907C020020FBAA000010B57E20FDF70CFE3F
S31508006FA0FBF774FE0B490C48018612213030FEF7B8
S31508006FB06EF8094930318884802107483030FBF75C
S31508006FC0FFFD7E20FDF7F8FD802103483030FBF7F2
S31508006FD003FE10BDFBAA00004C02002070B5044653
S31508006FE00D46E1B20548FDF727FB00BF012103481E
S31508006FF0FDF7C5FA0028F9D0204670BD00380140D3
S31508007000F0B587B000240020069005904049088B0B
S31508007010FAF73FFF07463F49FAF760FD05463C4940
S31508007020088BFAF736FF3B490490FAF757FD0746EF
S31508007030394801683846FAF710FD06462946FAF730
S315080070404DFD06903549C88CFAF723FF06463449A4
S31508007050FAF7FFFC054629460698FAF73FFD05901C
S3150800706030490598FAF7FDFC0546FAF754FF81B250
S315080070702748C183C08B00902548838B0022542162
S31508007080FE2000F0CEFE2249088BFAF702FF2049BF
S315080070900190C88BFAF7FDFE22490090FAF71EFD0B
S315080070A007460199FAF7DDFC06461A49FAF716FD6E
S315080070B017490390088BFAF7ECFE07461549FAF7C5
S315080070C00DFD0646144801683046FAF7C6FC0290DC
S315080070D00399FAF703FD05461149FAF769FC049086
S315080070E0FAF719FF84B20A48C08B0F49884204DBB5
S315080070F00748C08B0D49884204DD0222FE2157202D
S3150800710000F029FF054840384486204607B0F0BD00
S315080071107C02002000007A44900100200C04002024
S315080071200000C84100247449B80B00008813000009
S31508007130F0B587B000240020069005904049488B9A
S31508007140FAF7A7FE07463F49FAF7C8FC05463C4941
S31508007150488BFAF79EFE3B490490FAF7BFFC0746B0
S31508007160394801683846FAF778FC06462946FAF798
S31508007170B5FC06903549088CFAF78BFE0646344965
S31508007180FAF767FC054629460698FAF7A7FC05901C
S3150800719030490598FAF765FC0546FAF7BCFE81B250
S315080071A027488183C08B00902548838B0022542171
S315080071B0FE2000F036FE2249488BFAF76AFE20497F
S315080071C00190C88BFAF765FE22490090FAF786FC0B
S315080071D007460199FAF745FC06461A49FAF77EFC6E
S315080071E017490390488BFAF754FE07461549FAF7EC
S315080071F075FC0646144801683046FAF72EFC0290DC
S315080072000399FAF76BFC05461149FAF7D1FB049086
S31508007210FAF781FE84B20D48403804860848808B08
S315080072200D49884204DB0648808B0C49884204DDF8
S315080072300222FE21572000F08EFE204607B0F0BD40
S315080072407C02002000007A448C0100200C040020F7
S315080072500000C84100247449B80B000088130000D8
S31508007260F0B587B000240020069005904049488B69
S31508007270FAF70FFE07463F49FAF730FC05463C4940
S31508007280488BFAF706FE3B490490FAF727FC0746AF
S31508007290394801683846FAF7E0FB06462946FAF700
S315080072A01DFC06903549088CFAF7F3FD0646344965
S315080072B0FAF7CFFB054629460698FAF70FFC05901C
S315080072C030490598FAF7CDFB0546FAF724FE81B250
S315080072D027480184408C00902548038C01225421BC
S315080072E0FE2000F09EFD2249488BFAF7D2FD204980
S315080072F00190088CFAF7CDFD22490090FAF7EEFBCB
S3150800730007460199FAF7ADFB06461A49FAF7E6FB6E
S3150800731017490390488BFAF7BCFD07461549FAF753
S31508007320DDFB0646144801683046FAF796FB0290DC
S315080073300399FAF7D3FB05461149FAF739FB049086
S31508007340FAF7E9FD84B20A48008C0F49884204DB43
S315080073500748008C0D49884204DD0222FE21572089
S3150800736000F0F9FD054840380486204607B0F0BD10
S315080073707C02002000007A448C0100200C040020C6
S315080073800000C84100247449B80B000088130000A7
S3150800739070B5044600257E20FDF70EFCA34800883C
S315080073A040280ADD0020A1490880A1490870FF216C
S315080073B001319E48801DFAF7F0FA9D4800780300CF
S315080073C0FDF78BFC080521364760DAF1F0EF00205F
S315080073D0964948717E2C0FD108800120944908707F
S315080073E0924801880088401C904A1080901D445499
S315080073F000201146C87002E000208C490880002051
S315080074008A4908710FE1FE2C01D0002C0FD187485C
S3150800741001880088401C854A1080901D445402202B
S315080074208349087010460079001911460871FAE078
S315080074307E4801880088401C7C4A1080901D445470
S3150800744003207B4908701046007900191146087117
S31508007450E9E0764801880088401C744A1080901D2F
S3150800746044540420724908701046007900191146E0
S3150800747008710846C470C078002802D105206C49F6
S315080074800870D0E069484079012856D15E2C1CD195
S31508007490664800797E30654908717E21634802880E
S315080074A00088401C614B1880981D8154801FC07845
S315080074B0401EC0B21946C870002802DC05205C4987
S315080074C0087000205949487155E05D2C1CD1574871
S315080074D000797D30554908717D2154480288008815
S315080074E0401C524B1880981D8154801FC078401E3E
S315080074F0C0B21946C870002802DC05204C4908703D
S3150800750000204A49487136E0484800790019474939
S315080075100871084601880088401C444A1080901D5E
S315080075204454801FC078401EC0B21146C870002857
S3150800753021DC05203E4908701DE07D2C03D1012081
S315080075403A49487117E039480079001937490871EE
S31508007550084601880088401C344A1080901D44540F
S31508007560801FC078401EC0B21146C870002802DCD1
S3150800757005202F49087056E02C480079C043401C66
S31508007580C5B27D2D05D15D2C17D106202849087076
S3150800759013E07E2D08D15E2C0FD1062024490870F1
S315080075A00BE03FE02FE011E0A54203D10620204979
S315080075B0087002E007201E4908701C4801880088E8
S315080075C0401C1A4A1080901D44542CE01748018824
S315080075D00088401C154A1080901D44547E2C08D102
S315080075E001211448017100201146088010490870CD
S315080075F008E000200D49088000210E48017100208E
S315080076000B4908700FE000200949087007480188EF
S315080076100088401C054A1080901D445400201146DD
S31508007620088000E000BF00BF70BD0000A405002070
S31508007630F10100200C04002070B502460020134614
S315080076400C461D02FF26360235402543284670BDE6
S3150800765086B004460D4626686768A0680590E06807
S3150800766004902069039060690290A0690190E0691E
S31508007670009017A0FDF7F0FA31461BA0FDF7ECFACB
S3150800768039461CA0FDF7E8FA1DA00599FDF7E4FAAE
S315080076901EA00499FDF7E0FA1FA00399FDF7DCFA8E
S315080076A020A00299FDF7D8FA23A00199FDF7D4FA8C
S315080076B026A00099FDF7D0FA2948416A29A0FDF7C6
S315080076C0CBFA29462BA0FDF7C7FA00BFFEE7000054
S315080076D05B48617264206661756C742068616E64CB
S315080076E06C65725D0D0A00005230203D2025780D2C
S315080076F00A0000005231203D2025780D0A000000BE
S315080077005232203D2025780D0A0000005233203DD4
S315080077102025780D0A000000523132203D202578B8
S315080077200D0A0000537461636B6564204C52203D5A
S315080077302025780D0A000000537461636B65642088
S315080077405043203D2025780D0A00000053746163DC
S315080077506B656420505352203D2025780D0A0000A1
S3150800776000ED00E05343425F53484353523D2578AA
S315080077700D0A000043757272656E74204C52203DE6
S315080077802025780D0A0000000649074801860021D1
S31508007790303041805F218180C18001810021418193
S315080077A070470000FBAA00004C03002000B51549ED
S315080077B015480186FF210F31303041800A210181A9
S315080077C0A021C180C821818078214181B221C1814F
S315080077D032210182BE2181810C4901830B49253959
S315080077E04183052141820A218182C1820849818318
S315080077F0C183018441841221FDF749FC02493031D5
S31508007800888400BDFBAA00004C02002078210000F5
S315080078100410000010B57E20FDF7CEF9FEF7FAFE3B
S31508007820012800D110BD6048407901287ED15E4804
S315080078302030807E002802D0012860D137E0402120
S315080078405A48FBF7ABFB00281DD157482030407E2D
S31508007850012805D100205649486053492031487609
S315080078605348406D5349884220D2514840687D218B
S31508007870090188421AD24C4890384089002815D107
S31508007880FCF726FF12E048482030407E002803D146
S3150800789001204549203148764548C06E4549884209
S315080078A002D2FCF715FF01E0FDF704F879E040493C
S315080078B04868FF21F531FAF72DF8C007C00F0028F0
S315080078C00ED180210920C006FBF773FB012137483A
S315080078D0FBF76FFB10210920C006FBF76AFB0DE0DA
S315080078E080210920C006FBF762FB10210920C0068B
S315080078F0FBF75DFB01212D48FBF759FB51E02A48B0
S315080079002030807E052829D129494868FF21F5318C
S31508007910FAF700F8C007C00F002810D18021092007
S31508007920C006FBF746FB0121204800E03AE0FBF7DA
S3150800793040FB10210920C006FBF73BFB30E0802105
S315080079400920C006FBF733FB10210920C006FBF708
S315080079502EFB01211548FBF72AFB21E012482030AF
S31508007960807E06280ED180210920C006FBF71FFB62
S3150800797010210920C006FBF71AFB01210B48FBF76B
S3150800798016FB0DE080210920C006FBF712FB01213A
S315080079900648FBF70EFB10210920C006FBF709FB7A
S315080079A000BF00BF00BF3DE70C04002000040048EC
S315080079B00C02002030750000FCF702FAFBF748FDC0
S315080079C0FBF786FEFAF7FAFFFAF792FD0B20FAF7AD
S315080079D0C1FC0C20FAF7BEFC0920FAF7BBFC032011
S315080079E0FAF7B8FC01219348FAF728FE4B20000263
S315080079F0FAF74AFF0121904841710021C171002020
S31508007A008D492031C875887501218B488172FBF72D
S31508007A1053FDFCF70BFA1A216320FCF735FAFFF73A
S31508007A2059FAFCF70FFD00F0A1F983489038408910
S31508007A30002801D1FCF74CFE7F217E20FDF7FAF8DD
S31508007A4000217D48C17000207B4920318873EFE012
S31508007A507948C0780300FDF740F90805134D8B9E59
S31508007A60B1C4D7EAFAF712FEFFF7D4FEFDF726FFF0
S31508007A70FBF722FD01F0D8FC7E20FDF79DF8D6E045
S31508007A80002301221946184600F09AFC00231A46DC
S31508007A901946184600F094FC6848406868498842C8
S31508007AA004D908216748FBF782FA1DE0634948684C
S31508007AB0FF21F531F9F72EFFC007C00F00280ED1B8
S31508007AC080210920C006FBF772FA10210920C0069A
S31508007AD0FBF76DFA01215B48FBF769FA04E0102110
S31508007AE00920C006FBF765FAFAF77AFE7E20FDF74D
S31508007AF063F89CE0FAF7CAFDFBF7DEFC00230122D7
S31508007B001946184600F05CFC00231A461946184622
S31508007B1000F056FC494840684949884204D908217A
S31508007B204848FBF744FA1DE044494868FF21F53107
S31508007B30F9F7F0FEC007C00F00280ED180210920F2
S31508007B40C006FBF734FA10210920C006FBF72FFA06
S31508007B5001213C48FBF72BFA04E010210920C00656
S31508007B60FBF727FAFEF7E2FB7E20FDF725F85EE035
S31508007B70FDF7A0FA20210920C006FBF71AFAFAF742
S31508007B8085FDFFF747FEFDF799FEFBF795FC7E207E
S31508007B90FDF712F84BE0FDF71BFC20210920C00673
S31508007BA0FBF707FAFAF772FDFFF734FEFDF786FED4
S31508007BB0FBF782FC7E20FCF7FFFF38E0FDF77AFA38
S31508007BC020210920C006FBF7F4F9FAF75FFDFFF755
S31508007BD021FEFDF773FEFBF76FFC7E20FCF7ECFF3A
S31508007BE025E0FDF7F5FB20210920C006FBF7E1F9A2
S31508007BF0FAF74CFDFFF70EFEFDF760FEFBF75CFC9F
S31508007C007E20FCF7D9FF12E0FDF76EFD2021092042
S31508007C10C006FBF7CEF9FAF739FDFFF7FBFDFDF7CE
S31508007C204DFEFBF749FC7E20FCF7C6FF00BF00BFF0
S31508007C300EE70000002401400C0400200C0200207E
S31508007C40204E000000040048FEB546480088FAF7B2
S31508007C5020F90746444881693846FAF7D3F900D22D
S31508007C60FEBD414A11685068F9F7F3FE3E4988603F
S31508007C700A46D1689068F9F7ECFE02903A48C1685E
S31508007C8001208007F9F7EDFE0090374881680098D3
S31508007C90F9F7E3FE0746344801693846F9F788FEDE
S31508007CA00446314948690299F9F7DBFE01902E4AE4
S31508007CB091695069F9F7D5FE07462B48C1693846D8
S31508007CC0F9F70CFF0546284881682846F9F7C9FEE2
S31508007CD00546254A116A5069F9F7C3FE0746224840
S31508007CE081693846F9F7FAFE064621463046F9F71D
S31508007CF0B8FE064629460198F9F75AFE0746314660
S31508007D00F9F756FE184948622A20085EFAF7B6F8C7
S31508007D1000901548416A0098F9F74AFE0746FAF7AF
S31508007D20E1F800B2104948852A20085E898D884204
S31508007D3004DD0D48808D00B20B4948850A482A2182
S31508007D40415E002902DA0020074948850648C068CE
S31508007D500549086108468068C8600020014908800E
S31508007D6000BF7DE7500100204804002010B54021DF
S31508007D700F48F9F712FE40210D48FAF703FF0621CE
S31508007D800B48FDF784F90A49898988420AD10848C7
S31508007D903038008E0749884208D0FFF7F5FCFCF713
S31508007DA02BFF03E0FFF7F0FCFCF726FF10BD0000F1
S31508007DB07C030020FBAA0000F7B5A0B00C461546C8
S31508007DC080216846F9F7E9FD002700267E216846E6
S31508007DD00170FE214170EF2181700721C170209941
S31508007DE001710021417184712112C1710121017251
S31508007DF0457229128172012605E06846805DC01920
S31508007E00C7B2701CC6B20B2EF7DBF843401CC1B2D2
S31508007E106846C1727E2101730D21FCF77BFB23B0F6
S31508007E20F0BDFFB5A1B006461C462A9F802101A8D1
S31508007E30F9F7B3FD0020009000257E216846017100
S31508007E404671229981710721C17123990172002116
S31508007E50417284722112C17201210173477339126A
S31508007E608173012507E001A8415D00980818C0B292
S31508007E700090681CC5B20B2DF5DB0098C043401C6A
S31508007E80C1B26846C1737E2101740D2101A8FCF7B1
S31508007E9041FB25B0F0BDFFB585B005460E460E9FE1
S31508007EA000200190029003900490009000247E2107
S31508007EB068460171457186710421C171079901727D
S31508007EC00899417287723912C172012407E001A824
S31508007ED0015D00980818C0B20090601CC4B2082C56
S31508007EE0F5DB0098C043401CC1B2684601737E2189
S31508007EF041730A2101A8FCF70DFB09B0F0BD7FB557
S31508007F000446002000900190029003900026002568
S31508007F107E2168460170FE2141708F218170032100
S31508007F20C17000210171447121128171012505E09A
S31508007F306846405D8019C6B2681CC5B2072DF7DBD6
S31508007F40F043401CC1B26846C1717E210172092105
S31508007F50FCF7E0FA7FBDF7B584B005460E4600206B
S31508007F600090019002900390002700247E21684625
S31508007F700170467085700121C170694606980871BE
S31508007F80012405E06846005DC019C7B2601CC4B28A
S31508007F90052CF7DBF843401CC1B2684641717E21C7
S31508007FA081710721FCF7B6FA07B0F0BDF0B5ABB0A2
S31508007FB0074680210BA8F9F7F0FC002008900990E5
S31508007FC00A9005900690079000260490DFA004907A
S31508007FD0002400253B00FCF780FE06044BC3F1EFA6
S31508007FE0EEEDFBF717FA04460020089009900A9070
S31508007FF0E0B22104090E2202120E230E009201910C
S315080080000290D4A2092108A8FCF736FE7E2108A80A
S31508008010017300214173442181731321C173152211
S31508008020D1490CA8F9F7A0FC082208A90EA8033024
S31508008030F9F79AFCC5A0049005220CA80330049908
S31508008040F9F792FC012004E00BA9095C4919CDB2A5
S31508008050401C1728F8DBE843401CC1B210A8C170C1
S3150800806019267E21017119210BA8FCF753FA69E13B
S31508008070FBF7D0F904460020089009900A90E0B270
S315080080802104090E2202120E230E0092019102907B
S31508008090B0A2092108A8FCF7EFFDFBF7C1F90446D1
S315080080A00020059006900790E1B22004000E2202F7
S315080080B0120E230E009202910190A6A2092105A88C
S315080080C0FCF7DAFD7E2108A80173FE2141734421DD
S315080080D081733321C1733622A4490CA8F9F744FCED
S315080080E09AA0049005220CA803300499F9F73CFCE1
S315080080F096A00490052212A80499F9F735FC93A0D6
S315080081000490042213A803300499F9F72DFC0822D9
S3150800811008A90EA80330F9F727FC042110A8C17096
S31508008120082205A91330F9F71FFC082208A916A882
S315080081300330F9F719FC012004E00BA9095C491979
S31508008140CDB2401C3728F8DBE843401CC1B218A85A
S31508008150C1707E21017139210BA8FCF7DBF9F1E02A
S315080081607E2108A80173FE214173CF218173062160
S31508008170C1730021017475A0049005220CA8013072
S315080081800499F9F7F1FB012004E00BA9095C4919E8
S31508008190CDB2401C0A28F8D3E843401C0521490003
S315080081A00BAA50547E210B2011540C210BA8FCF766
S315080081B0B1F9C7E0C5E057E02BE0FFE77E2108A844
S315080081C00173FE214173CE2181730821C1730021F9
S315080081D0017467A0049007220CA801300499F9F7E6
S315080081E0C3FB012004E00BA9095C4919CDB2401C68
S315080081F00C28F8D3E843401CC1B20C200BAA115432
S315080082007E210D201154072041000BA8FCF782F9A6
S3150800821098E07E2108A80173FE214173CD21817360
S315080082200821C1730021017451A0049007220CA8EB
S3150800823001300499F9F798FB012004E00BA9095CC1
S315080082404919CDB2401C0C28F8D3E843401CC1B2EA
S315080082500C200BAA11547E210D2011540720410031
S315080082600BA8FCF757F96DE0FBF7D4F80446002095
S31508008270089009900A90E0B22104090E2202120E13
S31508008280230E00920191029032A2092108A8FCF758
S31508008290F3FCFBF7C5F80446002005900690079006
S315080082A0E1B22004000E2202120E230E0092029161
S315080082B0019028A2092105A8FCF7DEFC7E2108A862
S315080082C00173FE214173CB218173002101740121C1
S315080082D041741EA0049005220CA803300499F9F7EE
S315080082E043FB0C260BA98819082205A9F9F73CFBBC
S315080082F008360BA98819082208A9F9F735FB0836A4
S31508008300301FC1B208A8C173C07BC01EC1B208A87D
S315080083108174012004E00BA9095C4919CDB2401CFF
S31508008320B042F8DBE843401C0BA98855701CC6B25E
S315080083307E208855701CC6B231460BA8FCF7EAF8B1
S3150800834000E000BF00BF2BB0F0BD00005350726FB5
S3150800835042000000252E3258252E3258252E325836
S31508008360252E325800000000A6010020BB0100207F
S31508008370425F5631305F3400F8B506460C46F9F7C9
S3150800838059FF051E0F4600D00120014349000B483E
S315080083904908411AC90F0DD0002E01D0012100E06D
S315080083A000210C4361004908401AC00F02D1012080
S315080083B0FCF7EEFC28463946F8BD00000000F07FC1
S315080083C00FB591B0002010900F900E900D900C9064
S315080083D0FE480078642803D0FD48407A642804D112
S315080083E00121FB482038017203E00021F8482038B3
S315080083F001721398002802D001287DD173E21498DF
S31508008400002803D10021F2482038C172F148C189F9
S315080084101298814203D1EF48C08A0F9001E00520E7
S315080084200F900F98052802DC05200F9004E00F989E
S31508008430322801DB05200F900F991298411A1198DE
S31508008440814222DDE2482038C07A002815D1E14869
S3150800845070384068DF497039C8611498012804D11A
S315080084600121DB482038C17256E01498002853D100
S315080084700021D7482038C1724EE0149800284BD105
S315080084800021D3482038C17246E00F991298411846
S315080084901198814240DCCE482038C07A01283BD169
S315080084A0CB48C07A012831D1CA4870384068C949D2
S315080084B07039C969401AC84988420DD2C448B038CB
S315080084C00089462822DDC248B0380089801E81B25C
S315080084D0BF48B038018119E0BE4870384068BD49C8
S315080084E07039C969401A7D21890188420ED9B84870
S315080084F0B03800895F2800E0FEE307DAB448B038F0
S315080085000089801C81B2B248B03801810121B04887
S31508008510C17200212038C172AD482038C07A0128BE
S315080085207ED1AB48807E042803D0A948807E0528E2
S3150800853004D1002201210846FEF712F80F99129875
S31508008540411A119881426CDDA248703840687D2135
S31508008550C900884207D264209C49087000219C48BB
S3150800856020388173B8E19A482038807B00286DD17D
S3150800857001219748203881739648808964285CDAF7
S3150800858093486038018E408F081A81B29048603847
S315080085908187808F0990F9F77CFC01460A908F48FD
S315080085A00068F9F79BFA0B90F9F7E8FC8C4A03C2C6
S315080085B087482038008840430990F9F771FC0B91E9
S315080085C00A9087480CC80A98F9F778FB844A03C2C8
S315080085D0834903C9FFF7D0FE0B910A90F9F7F6FC19
S315080085E0804908607A48203800880890F9F751FCD5
S315080085F0014609907B480068F9F770FA7A490A90AB
S31508008600F9F72FFA0B90F9F786FC784908700846AF
S31508008610007864280DDC71480068F9F7AFFC01E0C2
S3150800862057E16CE00022724B0B910A90F9F7BAFCFD
S3150800863006D864206D49087002E064206B4908700A
S3150800864063486038018E4030C18245E16148703820
S31508008650806C7D21C90088424CD900205D4970395B
S3150800866088646248007864283FDA59486038018E81
S315080086704030C08A814233DD0121890757480068A6
S31508008680F9F796F90B90F9F746FC81B2504860382D
S31508008690028E4030C08A101A814205DA53480078A3
S315080086A0801E5249087020E049486038018E4030E3
S315080086B0C08A081A0A90F9F7E1FB0B904748016847
S315080086C00B98F9F79FFC10D248480078801C474958
S315080086D0087008460078642807DD6420087004E0FE
S315080086E042480078401D4149087039486038018E73
S315080086F04030C1823D48007834490870ECE034487F
S31508008700C07A002876D133488089642803DB642040
S315080087102E490870E0E02F48703840687D21C9006E
S31508008720884207D264202949087000212848203841
S315080087308173D1E026482038807B002874D1012136
S3150800874023482038817323488089642863DA2048BF
S315080087506038018E408F081A81B21D4860388187BB
S31508008760808F0990F9F795FB01460A901B48006827
S31508008770F9F7B4F90B90F9F701FC194A03C2144842
S315080087802038008840430990F9F78AFB0B910A9034
S3150800879013480CC80A98F9F791FA114A03C2104906
S315080087A003C9FFF7E9FD0B910A90F9F70FFC0D498C
S315080087B008600748203800880890F9F76AFB0146E0
S315080087C0099008480068F9F789F914E0F2000020D2
S315080087D02C0400207C02002070170000D400002022
S315080087E0D8000020E00000200000C842F100002068
S315080087F00000F03F67E0FE490A90F9F732F90B905E
S31508008800F9F789FBFB49087008460078642805DDF6
S315080088106420087002E06420F6490870F648018E64
S315080088204030C18258E0FFE7F448806C7D21C900DA
S31508008830884243D90020F1498864EF48018E4030C8
S31508008840C08A814231DD01218907ED480068F9F7C0
S31508008850AFF80B90F9F75FFB81B2E748028E40301C
S31508008860C08A101A814205DAE2480078801EE1497A
S3150800887008701FE0E048018E4030C08A081A0A9046
S31508008880F9F7FCFA0B90DE4801680B98F9F7BAFB82
S3150800889010D2D8480078801CD64908700846007857
S315080088A0642807DD6420087004E0D2480078401D7B
S315080088B0D0490870D048018E4030C182CD48007832
S315080088C0D049087008E0CC485038007ACD4908707D
S315080088D002E00020CB490870CA4802781499139818
S315080088E0FDF73EFE08E21498002803D10021C2488D
S315080088F040300173C0486030807E012804D00228C9
S315080089007ED003287DD199E0BC4870304188129802
S31508008910814204D1B9487030408A0F9001E00A209C
S315080089200F90B64840687D21C900884277D3B2487F
S315080089304030407B002872D1AF484030018881839F
S3150800894001214173808B0A90F9F7A3FAAE490B907F
S31508008950F9F758FB1AD8A8484030808B0790F9F7E2
S3150800896098FA01460890A948F9F7B8F8A84909906D
S31508008970F9F777F8A7490A90F9F71AF80B90F9F773
S31508008980CAFAC1B29C48603081723FE09A484030CA
S31508008990808BFF210A3188421ADC97484030808B49
S315080089A00790F9F776FA014608909748F9F796F886
S315080089B097490990F9F755F896490A90F8F7F8FF94
S315080089C00B90F9F7A8FAC1B28B48603081721DE0A6
S315080089D089484030808B0790F9F75BFA0146089082
S315080089E08948F9F77BF88C490990F9F73AF88949E3
S315080089F00A90F8F7DDFF0B90F9F78DFAC1B202E09D
S31508008A000EE029E00BE07C48603081727A486030DD
S31508008A10807A642803DB642177486030817229E014
S31508008A207648703041881298814204D17348703074
S31508008A30408A0F9001E00A200F901BE06F487030C3
S31508008A4081881298814204D16C487030808A0F90D0
S31508008A5001E00A200F900DE068487030818812986E
S31508008A60814204D165487030808A0F9001E00A205F
S31508008A700F9000BF00BF0F98052802DC05200F9055
S31508008A8004E00F98322801DB32200F905A486030F4
S31508008A90007B002802D11198FDF706FD0F99129860
S31508008AA0411A119881422ADB5448406853490862A2
S31508008AB000208863C86350491198C8870846403023
S31508008AC0007B00280FD11498012807D11E214A4897
S31508008AD0603001720121203801730BE000214648FD
S31508008AE04030017306E01498002803D1002142485B
S31508008AF040300173002140484030417241E10F99EE
S31508008B001298411811988142F8DC3B484030007BA6
S31508008B10012809D100213848403001733748406898
S31508008B20364908620020886333486030007B002895
S31508008B30E4D132487030408A0A280BDB2F48406A55
S31508008B400A90F9F7A6F935490B90F8F7C7FF3449A3
S31508008B50086020E029487030408A0A2810DA274839
S31508008B607030408A07280BDD2448406A0A90F9F7D6
S31508008B7090F92C490B90F8F7B1FF294908600AE0EB
S31508008B801E48406A0A90F9F784F927490B90F8F7C6
S31508008B90A5FF2349086018484030008B0890F9F76C
S31508008BA078F90A9014484030008B0790F9F771F964
S31508008BB008901B4801680898F8F753FF09900A9926
S31508008BC0F8F74FFF0B90F9F7D9F9184A03C20A4884
S31508008BD06030807A401D0590F9F762F9099108908E
S31508008BE005484030008B0190F9F76EF905911FE0B2
S31508008BF00000C842F1000020CC0300200C0200202F
S31508008C00D4000020F200002000007A4300008243CE
S31508008C100000BE42000040400000B44200803B45D0
S31508008C20CC0000200000FA440080BB44E800002085
S31508008C300490FB4903C9FFF79FFB03910290059B2C
S31508008C40049AF9F7A3F807910690099B089AF9F789
S31508008C5035F80B910A90F9F773F981B2F1488180DA
S31508008C60FF387138806A0A90F9F713F9EE490B90C4
S31508008C70F8F734FFED490860EA489030408B0890D1
S31508008C80F9F707F90A90E7489030408B0790F9F70B
S31508008C9000F90890E54801680898F8F7E2FE099097
S31508008CA00A99F8F7DEFE0B90F9F768F9DC4A03C271
S31508008CB0DC48B030807A401D0590F9F7F1F8099143
S31508008CC00890D8489030408B0190F9F7FDF8059147
S31508008CD00490D34903C9FFF74FFB03910290059B04
S31508008CE0049AF9F753F807910690099B089AF8F73A
S31508008CF0E5FF0B910A9000E01BE2F9F721F981B232
S31508008D00C848C180FF3801388089642827DAC848EE
S31508008D1080890890F9F7BDF80A90C5487038406B05
S31508008D200590F9F7B6F8C3490690F8F7D7FE089004
S31508008D30BF484188FF305130008F081A0690F9F76E
S31508008D409DF807900899F8F7C9FE09900A99F8F767
S31508008D5088FEB9490B90F8F7C1FEB8490860B148D2
S31508008D608088642802DB6421AE488180AD48C088CB
S31508008D70642802DB6421AB48C1800121A948B030D0
S31508008D800173A8489030007B00287AD0012879D151
S31508008D90A448B030007AAA49097888420EDA002138
S31508008DA0A048B0300172203801730020A0497039FC
S31508008DB0C86400219B48B030417260E10F9912984F
S31508008DC0411A119881420EDD96489030407B012861
S31508008DD004D19448B030817A417250E164219148B7
S31508008DE0B03041724BE18F48B030807E0300FBF70C
S31508008DF074FF06FD04098DFCFBFD8A48B030817AB4
S31508008E0041723BE18A487038806B89497039C96B71
S31508008E10401A7D21C90088424DD985487038806B33
S31508008E2083497039C8637F485030C18F1198814291
S31508008E300CDD7C4880880A3081B27A488180C088F7
S31508008E40642834DB64217748C18030E00F980B90A2
S31508008E5074485030C18F1198411A0B98C20F1018D8
S31508008E604010401C81420EDA6E488088801C81B210
S31508008E706C488180C088642819DB64216948C180F0
S31508008E8015E0FDE03AE10F980B9066485030C18F27
S31508008E901198411A0B98C20F10184010801C814275
S31508008EA005DD60488088801E81B25E4881805D4904
S31508008EB050311198C8875E48703840685C497039E7
S31508008EC0096A401A5F49884211DD56488088401D64
S31508008ED081B2544881808088642802DB6421514825
S31508008EE081805348703840685149703908624D4846
S31508008EF0B030007B002804D14A48B030817A4172EC
S31508008F0003E048480179B0304172B7E04848703804
S31508008F10806B47497039C96B401A7D21C900884260
S31508008F204BD943487038806B41497039C8633D480E
S31508008F305030C18F119881420CDD3A48C0880A30FA
S31508008F4081B23848C180C088642832DB642135483C
S31508008F50C1802EE00F980B9032485030C18F11987F
S31508008F60411A0B98C20F10184010401C81420CDAA7
S31508008F702C48C088801C81B22A48C180C0886428D1
S31508008F8017DB64212748C18013E00F980B9025480A
S31508008F905030C18F1198411A0B98C20F1018401003
S31508008FA0801C814205DD1F48C088801E81B21D488D
S31508008FB0C1801C4950311198C8871D4870384068CF
S31508008FC01B497039096A401A1F49884215DD154838
S31508008FD0C088401D81B21348C180C088642802DB5E
S31508008FE064211048C18002E034E00BE042E01048FA
S31508008FF0703840680E49703908620A488179B0307D
S3150800900041723BE007489030C07A01281ED1002003
S315080090100449B031487200210248B030017218E0A4
S31508009020E80000207C0300200000FA44CC00002061
S315080090307C02002000007A440000C842D4000020C8
S31508009040F200002088130000581B00001E203B4930
S31508009050487200BF39482038C07A012806D1002155
S315080090603648417200203549087202E01E2133480D
S31508009070417200BF32213148417200BF00BF41E052
S315080090802E48807E012829D10F99129841181198E7
S3150800909081421FDB2948B0380179B03041720F99F7
S315080090A012984018801E119988420FDD24480078CE
S315080090B0002822D12148B0388088401D81B21F4837
S315080090C0B038818001201E49087016E000201C492E
S315080090D0087012E00021194841720EE01748807E98
S315080090E0042803D01548807E052803D1002013499B
S315080090F0487202E00A211148417203E000210F4834
S31508009100417200BF00BF0D48807E012808D10B4878
S31508009110407A02460B9014991398FDF721FA07E056
S315080091200648007A02460B9014991398FDF718FA28
S3150800913000BF00BF109815B000BD00002C04002029
S31508009140F000002010B5002201210846FDF708FAB4
S315080091504C49088CF8F79DFE4B490860FEF774FDEC
S3150800916048482030407C002839D14848464948605C
S315080091704448008CB42807D04248008CB32803D052
S315080091804048008CB52804D101203E492031C874D6
S3150800919003E000203B492031C8743D48406E3D49F4
S315080091A0884267D93748408C801E3B4909888842DF
S315080091B00DDC3448408C801C37490988884206DB18
S315080091C0FDF7B6FF01202F492031487403E02D48EA
S315080091D0408C3149088000202D4948664AE02948D4
S315080091E02030407C01283BD12C4827494860254837
S315080091F0008CE62809D02348008CFF212C318842B0
S3150800920003D02048008CE72804D101211D482030CE
S31508009210C17403E000201B492031C8741C48406E05
S315080092201C49884226D91748408C801E1A49098845
S3150800923088420DDC1348408C801C174909888842EF
S3150800924006DBFEF70DF802200E492031487403E0CC
S315080092500C48408C1049088000200D49486609E0F2
S3150800926000200B494866084948850122FE215720F7
S31508009270FEF771FE0448408DC2B201210020FDF7B9
S315080092806FF910BD0C040020480400200000344388
S315080092900C0200208813000000010020000066432D
S315080092A030B503465A480068181AFF24F534A04218
S315080092B001D957480360481E904248DD5548007852
S315080092C0002816D1881A3C2805DA881A3C24201A60
S315080092D0514C207002E000204F4C20704E48007818
S315080092E05524201A4C4C2070204600784B4C207090
S315080092F02AE04B480078002822D14A480088401ABC
S3150800930007280ADD454C2078C40F24186410424DFE
S315080093102C7028460078414C207042480088401A34
S31508009320012808DD3D480078401E3C4C2070204648
S315080093300078394C20703B4802800120384C207058
S3150800934036480078344C2070364802805DE0481E66
S3150800935090424CDC481C824249DC2E4800780128A1
S3150800936028D12F48007800282AD12E480088801A4C
S3150800937007280BDD294C2078C40F24186410264DC5
S315080093802C7028460078254C20700DE0254800886A
S31508009390801A012808DB21480078401E1F4C2070DF
S315080093A0204600781C4C20701E48028001201C4C68
S315080093B0207005E017480078002801D1164C207067
S315080093C0481E904205D115480078401E124C207060
S315080093D01BE08A4205D111480078001F0E4C207008
S315080093E013E00E480078801F0B4C20700DE000201B
S315080093F0094C20700A4C20700120064C2070094840
S315080094000088824201DB074802800348007830BDA5
S3150800941004010020F80000200201002003010020BA
S315080094200A0100200801002010B5FDF7E1FA01281D
S315080094300AD1FE484068FF21F531884203D9042144
S31508009440FB48F9F7B4FD10BDFA48407900287DD1EC
S315080094500021F8482030017610210920C006F9F7C6
S31508009460A6FD80210920C006F9F7A1FD0121F048D3
S31508009470F9F79DFD0020EF49203188760023012267
S3150800948019461846FEF79CFF00231A461946184641
S31508009490FEF796FFE5484068FF21F531884209D274
S315080094A0E4482030C07D002803D10421E048F9F7BC
S315080094B080FDEDE20421DE48F9F779FD0020DD495B
S315080094C02031C875D9484068DB498842F1D9D9485E
S315080094D0807A002823D120210920C006F9F767FDE4
S315080094E0D24840687D214901884201D2FBF7B4F889
S315080094F00821CF48F9F75BFD0021CE48C17100204D
S31508009500CC492031C8720021CA4820300173002096
S31508009510C649486248637D204001486018E0C5484E
S315080095208079012814D10020C04948600021C1482B
S31508009530C1712030C17201730020BC49486248637A
S31508009540BC49203188760121BA4800E013E0417110
S315080095504021B748F9F722FD0028AAD02021092082
S31508009560C006F9F726FD0020B24920318876012188
S31508009570B04841718CE2AF482030807E0300FBF78B
S31508009580ACFB07057CE7F9F8F7F67B000021A9484C
S315080095900173C17201720020A4490864A5492031EB
S315080095A00876C87520210920C006F9F702FD0021B2
S315080095B0A0482030C172017300209C494862486364
S315080095C000219C4841730023012219461846FEF7DC
S315080095D0F7FE00231A4619461846FEF7F1FE954887
S315080095E04038418E0187418E8186018EC1868F481B
S315080095F040687D21090188422BD900208F490870CF
S3150800960040218B48F9F7CAFC00281AD110210920F5
S31508009610C006F9F7CCFC80210920C006F9F7C7FC7B
S3150800962001218348F9F7C3FCFBF716F8082180489F
S31508009630F9F7BDFC7E20FBF7BFFA1E20F9F77CF987
S3150800964002E000207949486004217948F9F7AFFC1F
S3150800965012E008217648F9F7ACFC74484068FF2107
S31508009660F531884208D9734890384089002803D1D3
S3150800967004216F48F9F79BFC09E26E484038018ED1
S31508009680C1866A484068FF21F531884204D2042120
S315080096906748F9F78EFC03E004216548F9F787FC6B
S315080096A0624948687D21C900F8F734F923282ED283
S315080096B05E4948687D21C900F8F72CF9192826D98A
S315080096C05C484038018EFF3851384088814207DAB5
S315080096D058484038418EFF385138408881420DDB62
S315080096E054482030007B012821D100204F4948608A
S315080096F0086202214F482030817618E000204B4945
S315080097004860086202204B49203188760FE04749B5
S3150800971048687D21C900F8F7FDF8232807D30020FB
S3150800972042494860086202214248203081763F4A11
S3150800973070325188FF325132508E01231A46FEF795
S315080097403FFE00231A4619461846FEF739FE9EE1E3
S3150800975038484038018EC18634484068FF21F531C3
S31508009760884208D204213248F9F723FC07E036E19B
S31508009770C8E07DE02BE004212D48F9F718FC2B48BA
S315080097804168703000897D22D2005043814210D250
S31508009790264A70325188FF325132508E01231A46BA
S315080097A0FEF70EFE00231A4619461846FEF708FE6F
S315080097B00CE000211F48017300201C494860012164
S315080097C01C48417203201B49203188765FE11948FD
S315080097D04038018EC186408EFF217D31884204DCE7
S315080097E014484038008E88420CDD002301221946B1
S315080097F01846FEF7E5FD00231A4619461846FEF7F1
S31508009800DFFD34E0094948687D21C900F8F782F888
S3150800981006497031498988421BD2044A70329188B8
S31508009820FF325132508E01231A4609E00C020020FD
S31508009830000400480C040020B80B0000C4000020F7
S31508009840FEF7BEFD00231A4619461846FEF7B8FD70
S315080098500DE09248018E4187002091494860002119
S315080098608E484030017304208C49603188760EE1B9
S315080098708A48408EFF217D31884203DC8748008E66
S3150800988088420CDD0023012219461846FEF798FD8A
S3150800989000231A4619461846FEF792FD31E080491C
S315080098A048687D21C900F8F735F87D497031098A7D
S315080098B00F3988421ED27A4A7032D189774A108E79
S315080098C001230022FEF77CFD74484030C07A012847
S315080098D006D10023012219461846FEF771FD10E04D
S315080098E06F4A7032D1886D4A508E01231A46FEF7A8
S315080098F067FD06E000206A4948600520674960312F
S315080099008876C4E066484068FF21F531884204D26B
S3150800991004216448F9F74DFB0FE061484068FF21D0
S31508009920F531884209D95E4840684B21C90088420A
S3150800993003D204215B48F9F73AFB594840685A496B
S3150800994088421ED2564A7032D189544A108E012353
S315080099500022FEF735FD51484030C07A012806D16D
S315080099600023012219461846FEF72AFD36E04C4A1E
S315080099707032D188494A508E01231A46FEF720FDD7
S315080099802CE004214748F9F714FB45484068464946
S31508009990C831884222D30020414948603F48603098
S315080099A0807D012804D106203C496031887605E08F
S315080099B000213A486030817620384171002301221F
S315080099C019461846FEF7FCFC00231A46194618469F
S315080099D0FEF7F6FC04213348F9F7E9FA57E00021C7
S315080099E02E4840300173C172017200202C49086468
S315080099F00865C864002129486030C17520210920FE
S31508009A00C006F9F7D6FA002024496031C8720873EF
S31508009A1023494862486300212048403041730023A7
S31508009A20012219461846FEF7CBFC00231A461946AA
S31508009A301846FEF7C5FC1948418E0187418E818676
S31508009A40018EC1864030C07900281FD1144840686D
S31508009A50164988421AD9FAF7FFFD002010494860CE
S31508009A600E4850384088032808DA0C48408E5A2891
S31508009A700CDC012009496031887607E00020074997
S31508009A8060318876002105484030417100BF00BF2B
S31508009A907E20FBF791F800BFD5E40000CC03002038
S31508009AA00C02002000040048A438000060EA000008
S31508009AB0D09A0008C800002044010000FC220008D3
S31508009AC0209B00080C020020A4080000804D000816
S31508009AD0015E2D01020304043506070809ACA24AF3
S31508009AE0041A5916011129250A450181580B1058DF
S31508009AF0594C4C3031313278010B11CB7E153E046E
S31508009B000132050513381206145941323030353200
S31508009B10384834353034324120041B7D5D7E0000E0
S705080018C515
